:020000040800F2
:1000000050570424AD02000889540008D74C00085A
:100010008554000899080008C38700080000000004
:100020000000000000000000000000003B5B000832
:10003000EF0A00080000000051550008CD5D0008DF
:10004000C7020008C7020008C7020008C70200086C
:10005000C7020008C7020008C7020008C70200085C
:10006000C7020008C7020008C7020008C70200084C
:10007000C7020008C7020008C7020008C70200083C
:10008000C7020008C7020008C7020008C70200082C
:10009000C7020008C7020008C7020008C70200081C
:1000A000C7020008C7020008C7020008C70200080C
:1000B000C7020008C7020008C7020008C7020008FC
:1000C000C7020008C7020008C7020008C7020008EC
:1000D000C70200083D6B0008C7020008C7020008FD
:1000E000C7020008C702000800000000C70200089D
:1000F000C7020008C7020008C7020008C7020008BC
:10010000C7020008C7020008C7020008C7020008AB
:10011000C7020008C7020008C7020008C70200089B
:10012000C7020008C7020008C7020008C70200088B
:10013000C7020008C7020008C7020008C70200087B
:1001400000000000000000000000000000000000AF
:10015000C7020008C7020008C7020008C70200085B
:10016000C7020008C7020008C7020008C70200084B
:10017000C7020008C7020008C7020008C70200083B
:10018000C7020008C7020008C7020008C70200082B
:10019000C7020008C7020008C7020008C70200081B
:1001A000C7020008C7020008C7020008C70200080B
:1001B000C7020008C7020008C7020008C7020008FB
:1001C000C7020008C7020008C7020008C7020008EB
:1001D000C70200088D540008C7020008C7020008C3
:1001E000C7020008C7020008C7020008C7020008CB
:1001F000C7020008C7020008C7020008C7020008BB
:10020000C7020008C7020008C7020008C7020008AA
:10021000C7020008C7020008C7020008C70200089A
:10022000C7020008C7020008C7020008000000005B
:10023000C7020008C702000800000000C70200084B
:10024000C7020008C7020008C7020008C70200086A
:10025000C7020008C7020008C7020008C70200085A
:10026000C7020008C7020008C7020008C70200084A
:10027000C7020008C7020008C7020008000000000B
:10028000C702000800000000C702000800000000CC
:1002900000000000C7020008DFF80CD000F050FAA0
:1002A00000480047AD930008505704240648804793
:1002B00006480047FEE7FEE7FEE7FEE7FEE7FEE74B
:1002C000FEE7FEE7FEE7FEE7D55D000899020008BD
:1002D0002DE9F05F0546002092469B46884606467B
:1002E000814640241BE0284641464746224600F00E
:1002F0005EF853465A46C01A914110D3114618462B
:10030000224600F045F82D1A67EB01084F462246B9
:100310000120002100F03CF817EB00094E41201E9F
:10032000A4F10104DFDC484631462A464346BDE8D5
:10033000F09F40EA01039B0703D009E008C9121FA0
:1003400008C0042AFAD203E011F8013B00F8013B8F
:10035000521EF9D27047421C10F8011B0029FBD134
:10036000801A704730B50B46014600202022012438
:1003700009E021FA02F59D4205D303FA02F5491B73
:1003800004FA02F52844151EA2F10102F1DC30BD89
:10039000202A04DB203A00FA02F100207047914045
:1003A000C2F1200320FA03F3194390407047202A3A
:1003B00004DB203A21FA02F00021704721FA02F30F
:1003C000D040C2F1200291400843194670472DE900
:1003D000FE4F804681EA0300C00F0C46009021F0DA
:1003E000004123F00045B8EB0200A94105D2404688
:1003F000214690461C460B46024623F0004010431F
:1004000047D0270DC7F30A00C3F30A510290401AE0
:10041000019040286BDAC3F3130040F4801B00986E
:10042000924620B10023D2EB030A63EB0B0B019839
:100430005946C0F140025046FFF7AAFF06460D4656
:1004400050465946019A00F08DF910EB08006141C1
:10045000002487EA115284EAE7731A4340D0009AD5
:1004600062B3019A012A4FEA075215DC001B61EBC7
:1004700002014FF0004202EA0752CDE90042001C9F
:1004800041F5801132462B4600F08DF903B0BDE8EE
:10049000F08F40462146F9E7001B61EB0201001C8A
:1004A00041F5801300185B412018A2F5001747EBB7
:1004B000030140EAD570B6196D4111E06D084FEAAD
:1004C000360645EAC0754FEA0752001B61EB020190
:1004D000001C41F5801149084FEA300000195141D4
:1004E00032462B4603B0BDE8F04F00F04DB90098FE
:1004F000012240000023D0EB020263EBE07300987E
:1005000021464FEAE074B8EB000061EB0401E9E733
:1005100083F000435BE781F0004158E72DE9FE4F8F
:1005200081EA030404F0004421F0004100944FF0FC
:10053000000B23F0004350EA01045ED052EA0304AA
:100540005BD0C3F30A54C1F30A552C44A4F2F3342C
:100550000194A0FB0254C1F3130141F48011C3F3D1
:10056000130343F4801301FB024400FB034E840A8F
:10057000970A44EA815447EA8357A4FB0768029527
:100580008D0A05FB07854FEA932C04FB0C542705C5
:10059000029D4FEA065847EA1637B5EB08056EEBA1
:1005A000070C870E920E47EA811742EA8312A7FBD7
:1005B0000201B6EB0B0164EB00042B0D43EA0C3394
:1005C0005E1844EB1C50DA465146E7FB0201C5F3C6
:1005D00013044FEA0B3343EA14534FEA0432019CED
:1005E00043EA0603A4F10C040294009CCDE900B494
:1005F00000F0D9F803B0BDE8F08F00200146F9E71C
:100600002DE9F04D81EA030404F0004B21F0004590
:1006100014464FF0000A23F0004150EA050220D0B2
:1006200054EA01021DD0C5F30A570246C5F313036D
:10063000C1F31300C1F30A5640F4801543F480134C
:10064000A7EB0608101BD64608F2FD3873EB050031
:1006500002D308F1010801E092185B41B8F1000FE4
:1006600003DA00200146BDE8F08D00204FF4801130
:10067000064684460EE0171B73EB050705D3121BD5
:1006800063EB050306434CEA010C49084FEA3000CE
:1006900092185B4150EA0107EDD152EA030012D0F3
:1006A00082EA040083EA0501084305D0101BAB4130
:1006B00006D20122002306E000224FF0004302E0B0
:1006C0006FF0010253101AEB06004CEB085110EBCF
:1006D0000A0041EB0B01BDE8F04D00F055B8C1F345
:1006E0000A52C1F3130140F2FF3341F480119A42E0
:1006F00002DA00200146704740F233439A42A2F2E8
:10070000334202DC5242FFF752BEFFF741BE000007
:1007100030B5041E71F1000404DB4FF00044404288
:1007200064EB0101141E73F1000405DB1C464FF05D
:100730000043524263EB0403994208BF904230BD2C
:10074000064C074D06E0E06840F0010394E807001E
:1007500098471034AC42F6D3FFF7A2FDB4BB0008B3
:10076000D4BB0008202A06DBCB17203A41FA02F05E
:1007700043EAE07306E041FA02F3D040C2F12002FE
:10078000914008431946704710B5141E73F10004D8
:1007900008DA401C41F1000192185B411A4301D173
:1007A00020F0010010BD2DE9F04D92469B4611B19D
:1007B000B1FA81F202E0B0FA80F220329046FFF7FF
:1007C000E7FD04460F4640EA0A0041EA0B015346A2
:1007D0005A46084313D0114653EA010019D0C8F114
:1007E00040025046FFF7E3FD05460E465046594687
:1007F0004246FFF7CDFD084305D0012004E0204626
:100800003946BDE8F08D0020054346EAE0762C43EA
:1008100037430A986305E40AA0EB08000022FD0AAA
:1008200044EA47540A3002D500200146E9E70105B1
:1008300010196941DDE9084500196941BDE8F04D2D
:10084000A2E770B58C1810F8015B15F0070301D111
:1008500010F8013B2A1106D110F8012B03E010F823
:10086000016B01F8016B5B1EF9D12B0705D4002346
:10087000521E0DD401F8013BFAE710F8013BCB1AE8
:10088000921C03E013F8015B01F8015B521EF9D5DD
:10089000A142D8D3002070BD00BFFEE770B5054669
:1008A0000C461646042D15D007DC7DB1012D0ED067
:1008B000022D0DD0032D50D10BE0202D0BD0212D7A
:1008C00030D0222D47D0232D47D145E046E045E0EA
:1008D00044E043E042E02078617840EA0120A178DA
:1008E00040EA0140E17840EA01601E490860207951
:1008F000087160794871A0798871084601791AA059
:1009000007F0B6FF174841791DA007F0B1FF154861
:10091000817922A007F0ACFF1248016826A007F0F9
:10092000A7FF1BE00F48007820700E480088000ADF
:1009300060700C480068000CA0700A480068000E47
:10094000E0700848007920710648407960710548D8
:100950008079A07102E001E000E000BF00BF00204C
:1009600070BD0000840100246C696E65636F64696A
:100970006E672E666F726D61743A25640D0A000011
:100980006C696E65636F64696E672E7061726974FD
:1009900079747970653A25640D0A00006C696E659A
:1009A000636F64696E672E64617461747970653A0F
:1009B00025640D0A000000006C696E65636F646950
:1009C0006E672E626974726174653A25640D0A005F
:1009D0000020704710B50349034806F0D1F9002004
:1009E00010BD00006C0C0024E801002470B5054621
:1009F0000C462846216804F0DDFE044806F09CF908
:100A00002846216807F0E0FE002070BDE8010024C0
:100A100010B504F043FF04F0F3FE0348006840F013
:100A200004000149086010BD9CEF00E02DE9F04191
:100A300080460D4616461F46002419E004EB0410BC
:100A40000D4911F81000B04210D104EB041001EB75
:100A500040004078B84209D104EB04100A4602EB8A
:100A60004000811C2A46404600F036F8601C84B2E3
:100A7000382CE3DBBDE8F081F8B000082DE9F04147
:100A800080460D4616461F4600241FE004EB8400F6
:100A900000EB44100F4911F81000B04214D104EBE0
:100AA000840000EB441001EB40004078B8420BD1C9
:100AB00004EB840000EB44100A4602EB4000811C6A
:100AC0002A46404600F008F8601C84B2092CDDDBA1
:100AD000BDE8F081CEB8000810B5002304E011F89D
:100AE000014B00F8014B5B1C9342F8D310BD7047DB
:100AF0002DE9F04385B004460D4617461E460E48C4
:100B00000088001B1FFA80F80B484088401B1FFA22
:100B100080F900200949098810224B46CDE90127B8
:100B20000096CDE9031042462946204600F03CFAE3
:100B300005B0BDE8F0830000404D0424E20100242C
:100B40002DE9FF4704460D4616461F460B48008810
:100B5000001B1FFA80F809484088401B1FFA80F9E3
:100B6000002010214B464246CDE90071CDE90260DC
:100B70002946204605F044F8BDE8FF87404D04248F
:100B80002DE9FF4704460D4616461F460B480088D0
:100B9000001B1FFA80F809484088401B1FFA80F9A3
:100BA000002018214B464246CDE90071CDE9026094
:100BB0002946204605F024F8BDE8FF87404D04246F
:100BC0002DE9F04106460C46174601221103144850
:100BD00000F074FC052000F050FA032004F0D0FE71
:100BE000C4F3074004F0CCFEC4F3072004F0C8FEB1
:100BF000E0B204F0C5FE002505E0FF2004F0C0FED1
:100C00007055681C85B2BD42F7DB00224FF480515D
:100C1000034800F053FC052000F02FFABDE8F081F6
:100C2000000402582DE9F0470746884691461C46C5
:100C30003E78B9F1200F1ED009DCB9F10C0F0DD0B0
:100C4000B9F1100F0FD0B9F1180F20D10FE0B9F1A1
:100C5000300F14D0B9F1400F19D114E006FB04F0A5
:100C600000F5002515E00F4806FB040511E00E48CD
:100C700006FB04050DE00D4806FB040509E00C48E1
:100C800006FB040505E00B4806FB040501E0BDE892
:100C9000F08700BF224629464046FFF791FF00BF7C
:100CA000F5E7000000080800001208000026080010
:100CB00000480800009208002DE9FF5F82460F46B9
:100CC00098469AF800900AF1010082460478B9F13A
:100CD000810F06DB402C04DBFF2C02D0B9F1FF0FA3
:100CE0000DD14FF0000B06E0002007F8010B0BF1CF
:100CF00001001FFA80FBC345F6DBBDE8FF9F7F2C98
:100D000003DAA4F14000C4B202E0A4F14100C4B28D
:100D1000A9F1810000F0FF09BE2010FB094000FB93
:100D200008F502980C2806D0102807D0182808D0FB
:100D300020280CD108E00A482E1809E009482E188E
:100D400006E005F5ED1603E005F5601600E0D4E7D2
:100D500000BF424631463846FFF732FF00BFCCE7BE
:100D60000014090000DD110010B500F001F810BDFD
:100D700010B586B04FF6FF7004F00CF8002404E0C4
:100D800000200DF80400601CC4B2182CF8DB1122FE
:100D900000216846FFF714FF6B464FF4784210219C
:100DA0000846FFF7A5FE002404E000200DF804002B
:100DB000601CC4B2182CF8DB082214216846FFF727
:100DC000FFFE6B464FF4784220211020FFF790FE83
:100DD000002404E000200DF80400601CC4B2182CAC
:100DE000F8DB08221E216846FFF7EAFE6B464FF447
:100DF000784230211020FFF77BFE012008F098FA9E
:100E000006B010BD2DE9FF4FC1B080460D461C460F
:100E1000AB462046E31704EB5373DB1021464FEA41
:100E2000E47C04EB5C7C4FEAEC0CA4EBCC0CBCF156
:100E3000000F02D04FF0010C01E04FF0000C6344B2
:100E4000224604EBD27C4FEA6C0C03FB0CF39FB2FE
:100E50000C2C0CD0102C0AD0182C08D0202C06D02A
:100E6000302C04D0402C02D045B0BDE8F08F3B467A
:100E7000224601A94398FFF7D5FE00262FE001A8DE
:100E800010F806904FF0000A23E009F0800028B126
:100E9000294640464E9A04F005F806E0509820B9DD
:100EA000294640464F9A03F0FDFF4FEA49604FEA5A
:100EB0001069681C85B2A5EB0B00A04205D15D4608
:100EC00008F101001FFA80F806E00AF101001FFA9C
:100ED00080FABAF1080FD8DB00BF701C86B2BE42A0
:100EE000CDDB00BFC0E72DE9FF4FA1B080460D4626
:100EF0001C46AB462046E21704EB5272D210214644
:100F0000E31704EB5373DB10A4EBC3030BB1012312
:100F100000E000231A44624397B20C2C08D0102C36
:100F200006D0182C04D0202C02D025B0BDE8F08FBC
:100F30003B46224601A92398FFF7BEFE00262FE07C
:100F400001A810F806904FF0000A23E009F0800095
:100F500028B1294640462E9A03F0A4FF06E03098B7
:100F600020B9294640462F9A03F09CFF4FEA49607A
:100F70004FEA1069681C85B2A5EB0B00A04205D1B1
:100F80005D4608F101001FFA80F806E00AF1010051
:100F900000F0FF0ABAF1080FD8DB00BF701CC6B220
:100FA000BE42CDDB00BFC0E72DE9F04F85B007465C
:100FB0000D4691469A46DDE90F4B0E9EB8460495C4
:100FC0000020039052E0039888BB3078802802DD2F
:100FD000012003904AE004EBD47108EB0902A2EB74
:100FE0006101B94202DA281985B247460498504493
:100FF000001BA84200DA3CE030780D2804D1281903
:1010000085B24746761C0AE0DDE9111023463246D8
:10101000CDE900B1029029463846FFF7F3FE761C71
:10102000204604EBD07107EB61018FB21EE0FFE7B1
:101030000020039008EB0900001BB84202DA2819CF
:1010400085B2474604985044001BA84200DA10E0DD
:10105000DDE9110123463246CDE900B0029129466F
:101060003846FFF740FFB61C381987B230780028A1
:10107000A9D100BF05B0BDE8F08F002107E0002234
:1010800001E0531CDAB2642AFBDB4B1CD9B281426B
:10109000F5DB70472DE9F04705460C4690469A4629
:1010A00095F80090681C05460778B9F1810F06DBBA
:1010B000402F04DBFF2F02D0B9F1FF0F0AD1002629
:1010C00004E0002004F8010B701CC6B24645F8DBB2
:1010D000BDE8F087BAF10C0F06D0BAF1100F04D0BA
:1010E000BAF1180F0FD107E00DE03B464A464146E2
:1010F0002046FFF79BFC06E03B464A464146204619
:10110000FFF7BCFC00BF00BF00BFE1E770B50524DE
:1011100006250726344454B108220549204603F029
:10112000DCFD042202491031284603F0D6FD70BDD3
:101130006A01002410B504460CB9012010BD94F8D2
:101140003500022803D0802060650120F6E734498D
:101150002068884205D333492068884201D801209D
:1011600000E00020C0B1042084F835002C4920683C
:1011700088420AD32B492068884206D82068006834
:1011800020F001002168086048E02068006820F035
:1011900001002168086041E02068006820F00E002E
:1011A000216808601E49206888420AD31D492068CA
:1011B000884206D82068006820F001002168086095
:1011C00005E02068006820F0010021680860206EBA
:1011D000006820F48070216E086094F85C10012093
:1011E000884011490860D4E919104860E06E40B1A8
:1011F000E06E006820F48070E16E0860D4E91C1095
:10120000486000BF002084F8340000BF012084F84B
:101210003500206D10B12046216D884700208DE7F4
:1012200010000240B80402400454025870B504464D
:1012300000F04AF906462546681C10B104480078BB
:10124000054400BF00F040F9801BA842FAD370BDEE
:101250001C0000240348006840F0010001490860B8
:101260007047000020040058F8B502460B460021E4
:10127000002600240020824D00BFFCE0012707FA71
:1012800001F61F6807EA0604B4427CD15F68022FAA
:1012900002D05F68122F1AD14FEAD10C02F1200759
:1012A00057F82C004F074FEAD76C0F2707FA0CF7B7
:1012B000B8434FEA417C4FEADC6C1F6907FA0CF730
:1012C00038434FEAD10C02F1200747F82C00106890
:1012D0004FEA410C032707FA0CF7B8431F7907F0D0
:1012E00003074FEA410C07FA0CF7384310605F68B8
:1012F000012F08D05F68022F05D05F68112F02D040
:101300005F68122F17D190684FEA410C032707FA44
:101310000CF7B8434FEA410CDF6807FA0CF7384383
:101320009060506801278F40B8431F79C7F30017BA
:101330008F4038435060D0684FEA410C032707FACA
:101340000CF7B8434FEA410C9F6807FA0CF7384393
:10135000D0605F6807F08057B7F1805F95D100BF1C
:10136000484F3F6847F00207DFF818C1CCF800701B
:1013700067463F6807F00207009700BF00BF424F73
:101380004FEA910C00E075E057F82C008F074FEA08
:10139000177C0F2707FA0CF7B8433C4FBA4201D12C
:1013A00000272DE03A4FBA4201D1012728E0394FFA
:1013B000BA4201D1022723E0374FBA4201D10327B5
:1013C0001EE0364FBA4201D1042719E0344FBA4229
:1013D00001D1052714E0334FBA4201D106270FE0AF
:1013E000314FBA4201D107270AE0304FBA4201D14A
:1013F000082705E02E4FBA4201D1092700E00A274D
:101400004FEA817C4FEA1C7C07FA0CF738431E4FE9
:101410004FEA910C47F82C002868A0435F6807F456
:101420008037B7F5803F00D1204328606868A0432B
:101430005F6807F40037B7F5003F00D120436860CC
:101440004FF0B0473868A0435F6807F48017B7F5DE
:10145000801F00D120434FF0B04738607868A04328
:101460005F6807F40017B7F5001F00D120434FF065
:10147000B0477860491C1029FFF400AFF8BD0000A8
:1014800080000058F4440258080400580000025834
:101490000004025800080258000C025800100258BC
:1014A0000014025800180258001C0258002002586C
:1014B0000024025842694A40426170470AB10183E0
:1014C00000E0418370470000014800687047000059
:1014D00014000024034800680349097808440149BE
:1014E00008607047140000241C00002410B503207D
:1014F00000F0E2F8002000F007F808B1012010BD6C
:1015000000F08CF80020FAE770B504460E48007829
:101510004FF47A71B1FBF0F00C490968B1FBF0F5BA
:10152000284603F097F908B1012070BD102C07D2AE
:1015300000222146501E00F082F80548046001E0B8
:101540000120F2E70020F0E71C0000240000002446
:10155000180000244178154A11600178F9B1121D74
:1015600041681160017B0907C27A41EA0261827A0F
:1015700041EAC241427B41EA8241827B41EA4241E7
:10158000C27B41EA0241427A41EA0221027A41EAFF
:10159000420102781143054A0832116005E000213A
:1015A000024A121D1160121D1160704798ED00E093
:1015B00000BF00BF00BFBFF35F8F00BF00BF00BF11
:1015C0000548006820F48030034908600020024983
:1015D000703108607047000024ED00E040F0010128
:1015E0000D4A11600C497039096841F480310A4A8A
:1015F000703A116000BF00BF00BFBFF34F8F00BF44
:1016000000BF00BF00BF00BF00BFBFF36F8F00BFB0
:1016100000BF00BF7047000094ED00E07047014636
:101620000846002809DB00F01F0301229A40430905
:101630009B0003F1E023C3F8002100BF70472DE9B0
:10164000F05F80460D46164607F034F907463946E6
:101650002A46334601F00700C0F1070ABAF1040F29
:1016600002D94FF0040A01E0C0F1070AD14600F1A7
:10167000040ABAF1070F02D24FF0000A01E0A0F10C
:10168000030AD4464FF0010A0AFA09FAAAF1010A3C
:101690000AEA020A0AFA0CFA4FF0010B0BFA0CFBE9
:1016A000ABF1010B0BEA030B4AEA0B04214640465F
:1016B00007F008F9BDE8F09F00BF00F00702064BF5
:1016C00019684FF6FF031940044B0B4343EA02210C
:1016D000014B196000BF70470CED00E00000FA05F7
:1016E000024611680120C2F8F803886B40F400300C
:1016F0008863886B40F48020886300207047000076
:1017000001460A680120C1F8F403002081F8EC03C7
:10171000906940F000609061506D024B1843506535
:1017200000207047030000107047024610684162B5
:1017300000207047F0B503461446002500221868C3
:10174000426A21B942EA04401E68B06219E0186892
:10175000806A02EB1042002508E0186800F58270EC
:1017600050F8250002EB1042681CC5B2481EA84282
:10177000F3DC42EA0447186800F582704E1E40F818
:1017800026700020F0BD000010B50446012003497A
:101790000870D4F8FC0305F013FE10BD31010024DD
:1017A00070B504460D46C5EBC50304F1380101EBE5
:1017B0008301CA682946D4F8FC0305F051FD70BDC9
:1017C00070B504460D46C5EBC50304F5FC7101EB8D
:1017D0008301CA682946D4F8FC0305F0AEFD70BD4C
:1017E00010B5044600200549087005A007F040F830
:1017F000D4F8FC0305F0E7FD10BD00003101002422
:101800005553422044657669636520446973636F6C
:101810006E6E65637465642E0D0A000070B5044633
:101820000D46002605F08000802808D105F07F00D5
:10183000C0EBC00104F1380000EB810607E005F0C1
:101840007F00C0EBC00104F5FC7000EB810605F0E1
:101850007F00307005F08000C009707000BF94F800
:10186000B803012801D1022070BD012084F8B8031B
:1018700000BF3146206806F06FFA00BF002084F8F0
:10188000B80300BF00BFEFE770B504460D46002661
:1018900005F08000802808D105F07F00C0EBC00172
:1018A00004F1380000EB810605E0C5EBC50104F545
:1018B000FC7000EB81060020B07005F07F003070F6
:1018C000C5F3C010707000BF94F8B803012801D1AF
:1018D000022070BD012084F8B80300BF31462068A3
:1018E00006F084FC00BF002084F8B80300BF00BFEE
:1018F000EFE7024601F00F00C0EBC00302F5FC70F9
:1019000000EB8300008B80B270472DE9F04705465D
:101910000E4690461F464FF00009002406F0800056
:10192000802808D106F07F00C0EBC00105F1380027
:1019300000EB810407E006F07F00C0EBC00105F575
:10194000FC7000EB810406F07F00207006F0800040
:10195000C0096070C4F80880E770607808B120782A
:10196000E080022F01D10020207100BF95F8B8035C
:10197000012802D10220BDE8F087012085F8B803D4
:1019800000BF2146286806F005F900BF002085F851
:10199000B80300BF4846EEE72DE9F04104460E4685
:1019A00017469846002506F07F00C0EBC00104F5FD
:1019B000FC7000EB8105EF60C5F814800020A86181
:1019C000687006F07F0028702069012800D12F611F
:1019D00006F07F0028B9227C2946206806F00CFB1F
:1019E00004E0227C2946206806F08AFC0020BDE83D
:1019F000F08170B504460D46002605F08000802871
:101A000008D105F07F00C0EBC00104F1380000EB05
:101A1000810605E0C5EBC50104F5FC7000EB81060D
:101A20000120B07005F07F003070C5F3C0107070F9
:101A300000BF94F8B803012801D1022070BD012035
:101A400084F8B80300BF3146206806F013FC05F0A7
:101A50007F0028B9217C04F56F72206806F0A4FB92
:101A600000BF002084F8B80300BF00BFE6E72DE9FF
:101A7000F04104460E4617469846002506F07F00C2
:101A8000C0EBC00104F1380000EB8105EF60C5F840
:101A900014800020A8610120687006F07F00287083
:101AA0002069012800D12F6106F07F0028B9227C2F
:101AB0002946206806F0A0FA04E0227C2946206826
:101AC00006F01EFC0020BDE8F08100002DE9FC5F5F
:101AD000044626684FF0000B002001908046002548
:101AE000009081468246FE4F206806F0C9FD00281E
:101AF0007DD1206806F0FCFD08B9BDE8FC9F206898
:101B000006F0F6FD00F00200022801D121684861CC
:101B1000206806F0EDFD00F40020B0F5002F67D13D
:101B20000025206806F0BAFD0190A8E0019800F0B9
:101B3000010000287ED0E9B2206806F0CEFD804684
:101B400008F00100002860D0012106F5306000EBAC
:101B500045108160306CE34988420ED3206901282A
:101B60000BD1D6F8080B00F4004030B14FF400411F
:101B700006F5306000EB45108160206901282BD10B
:101B8000C5EBC50104F5FC7000EB8100816806F52A
:101B9000306000EB45100069C0F31200091AC5EB74
:101BA000C50204F5FC7000EB82008161C5EBC50144
:101BB00004F5FC7000EB8100C5EBC502C16804F5BB
:101BC000FC7000EB820080680144C5EBC50204F59F
:101BD000FC7000EB8200C160E9B22046FFF7F0FD27
:101BE0002069012811D185B9C5EBC50101E0EEE2FC
:101BF00049E004F5FC7000EB8100406928B904F568
:101C00006F720121206806F0CFFA08F0080008285A
:101C10001DD1306CB349884210D3206901280DD101
:101C2000D6F8080B00F4004040B14FF4004106F52F
:101C3000306000E01FE000EB45108160204600F0BE
:101C40006DFC082106F5306000EB4510816008F05E
:101C50001000102805D1102106F5306000EB45106A
:101C6000816008F02000202805D1202106F5306091
:101C700000EB451081606D1C0198400801900198AF
:101C800000287FF453AF206806F032FD00F4802076
:101C9000B0F5802F7DD1206806F0F7FC019000257B
:101CA00085E0019800F0010000287CD0E9B22068AE
:101CB00006F0FDFC804608F00100E8B30120A840D2
:101CC000009040F6340080590099884340F6340172
:101CD0008851012106F5106000EB451081602069F4
:101CE000012815D1C5EBC50104F1380000EB8100D6
:101CF000C5EBC502C16804F1380000EB82008068C2
:101D00000144C5EBC50204F1380000EB8200C1605C
:101D1000E9B22046FFF744FD2069012810D15DB9E2
:101D2000C5EBC50104F1380000EB8100406918B92A
:101D300004F56F72012100E002E0206806F034FA39
:101D400008F00800082805D1082106F5106000EB0E
:101D50004510816008F01000102805D1102106F50B
:101D6000106000EB4510816008F04000402805D16C
:101D7000402106F5106000EB4510816008F002007C
:101D8000022805D1022106F5106000EB45108160A4
:101D900001E010E007E008F08000802803D1294628
:101DA000204603F07BFB6D1C0198400801900198D0
:101DB00000287FF476AF206806F09AFC00F000401F
:101DC000B0F1004F1AD140F60400805920F0010113
:101DD00040F60400815194F8EC03012807D100205B
:101DE00084F8EC0300212046FFF79EFC02E0204629
:101DF00000F060FB4FF0004021684861206806F069
:101E000077FC00F40060B0F5006F0CD140F60800DC
:101E1000805900F0010010B1204600F093FB4FF410
:101E2000006021684861206806F062FC00F00060F4
:101E3000B0F1006F17D14FF000602168486194F84D
:101E4000EC0368B9012084F8EC032068406DC0F30E
:101E50008300C4F8F00301212046FFF765FC02E08F
:101E6000204600F06FFB206806F042FC00F4805032
:101E7000B0F5805F60D140F60400805920F0010188
:101E800040F6040081511021206806F0BFFB4FF09E
:101E9000000B0CE0FF2106F5106000EB4B10816099
:101EA00006F5306000EB4B1081600BF1010B6068B0
:101EB0005845EFD84FF0FF3140F618008151001D12
:101EC000805940F0011140F61C008151206BA0B1F7
:101ED000D6F8840840F00B01C6F8841804E000002E
:101EE0000084D7170A31544F40F64400805940F01F
:101EF0000B0140F6440081510EE040F61400805979
:101F000040F00B0140F614008151001F805940F051
:101F10000B014FF401608151D6F8000820F4FE60F7
:101F2000C6F80008217C04F56F72206806F03CF9C1
:101F30004FF4805021684861206806F0D9FB00F416
:101F40000050B0F5005F7AD1206805F085FE20686A
:101F5000C06820F470502168C860206806F06EFBED
:101F600058B90021E1604FF4007161612068C068D8
:101F700040F410502168C86082E00321E1604021F4
:101F8000616101F029FC07469248874209D39248D3
:101F9000874206D22068C06840F470502168C8604B
:101FA0006EE08D48874209D38C48874206D220686C
:101FB000C06840F460502168C86061E0874887428B
:101FC00009D38748874206D22068C06840F4505041
:101FD0002168C86054E08248874209D3814887421B
:101FE00006D22068C06840F440502168C86047E0CD
:101FF0007C48874209D37C48874206D22068C06863
:1020000040F430502168C8603AE07748874209D3ED
:102010007648874206D22068C06840F42050216884
:10202000C8602DE0714887420AD37148874207D2C1
:102030002068C06840F410502168C86020E026E0A5
:102040006B48874209D36B48874206D22068C06834
:1020500040F400502168C86012E06648874209D306
:102060006548874206D22068C06840F4E050216885
:10207000C86005E02068C06840F4C0502168C860AE
:10208000204600F0CBF94FF40050216848612068E9
:1020900006F02EFB00F01000102845D12068806962
:1020A00020F0100021688861D6F8209009F00F0018
:1020B000C0EBC00104F5FC7000EB810AC9F343409A
:1020C00002281AD147F6F07009EA000030B3C9F3CC
:1020D0000A123046DAF80C1006F010FBC9F30A11A8
:1020E000DAF80C000844CAF80C00C9F30A11DAF84F
:1020F00018000844CAF8180010E0C9F34340062845
:102100000CD1082204F56F71304606F0F7FAC9F3D6
:102110000A11DAF818000844CAF818002068806923
:1021200040F0100021688861206806F0E1FA00F0B4
:102130000800082805D1204600F0D0F908202168C1
:102140004861206806F0D4FA00F48010B0F5801FD2
:1021500007D1E9B2204600F051F84FF48010216811
:102160004861206806F0C4FA00F40010B0F5001FC2
:1021700007D1E9B2204600F04AF84FF40010216878
:102180004861206806F0B4FA00F08040B0F1804F5A
:1021900006D12046FFF7F8FA4FF0804021684861E9
:1021A000206806F0A5FA00F0040004280FD120688A
:1021B000D0F8049009F00400042802D12046FFF76B
:1021C0000FFB2068406840EA09002168486000BFB2
:1021D00093E40000C0ACD800C0E1E4000024F400A7
:1021E00080730601A0491A01002D310140A44C0161
:1021F00000366E0120ABA6010048E80170B5044628
:102200000D462946D4F8FC0305F042F970BD70B5BF
:1022100004460D462946D4F8FC0305F03CF970BD90
:1022200030B58BB00446002514B901200BB030BD89
:10223000032084F8B903204600F0A0F8206805F0D8
:10224000D3FE282204F110016846FEF772F894E8E4
:102250000F0005F023FD0021206806F063FA002539
:1022600030E00121C5EBC50204F1380000EB82002B
:102270004170C5EBC50204F1380000F82250C5EBEF
:10228000C50200EB8200C5800021C5EBC50204F148
:10229000380000EB8200C170C5EBC50204F13800C4
:1022A00000EB82008160C5EBC50204F1380000EB51
:1022B0008200C160C5EBC50204F1380000EB82006A
:1022C00041616D1C0F2DCCD3002536E00021C5EBFC
:1022D000C50204F5FC7000EB82004170C5EBC5023D
:1022E00004F5FC7000F82250C5EBC50204F138007B
:1022F00000EB8200C580C5EBC50204F5FC7000EB65
:102300008200C170C5EBC50204F5FC7000EB8200D1
:102310008160C5EBC50204F5FC7000EB8200C16072
:10232000C5EBC50204F5FC7000EB8200416120683A
:1023300000F5827040F825106D1C0F2DC6D32822A1
:1023400004F110016846FDF7F4FF94E80F0005F072
:1023500075FD012084F8B903A06A012802D1204646
:10236000FFF7CEF9606A012802D12046FFF7B8F9DD
:10237000206805F054FD002058E7000010B5B6B005
:1023800004464FF4802002904FF44010239002A89E
:1023900000F05EFB1E492068884235D100BF1D4811
:1023A000006840F001001B4908600846006800F022
:1023B0000100019000BF00BF4FF4C05031900220D7
:1023C000329000203390032034900A20359031A9B8
:1023D0001148FEF749FF00BF0E480838006840F07A
:1023E00000600C49083908600846006800F0006089
:1023F000019000BF00BF002201216520FFF71FF9F7
:102400006520FFF70CF900E000BF36B010BD0000FA
:1024100000000840E04402580000025870B504462D
:102420000125E06810B102280AD104E00CA006F0F2
:102430001FFA002509E011A006F01AFA012504E0B0
:1024400015A006F015FA012500BF00BFD4F8FC0363
:1024500005F044F82946D4F8FC0305F079F870BD7E
:1024600055534220446576696365204C6962726108
:10247000727920205B48535D0D0A000055534220BD
:10248000446576696365204C6962726172792020C7
:102490005B46535D0D0A0000555342204465766942
:1024A0006365204C69627261727920205B46533FFC
:1024B0005D0D0A0010B5044603A006F0D9F9D4F862
:1024C000FC0305F02DF810BD446576696365205264
:1024D0006573756D65640D0A0000000010B5044653
:1024E000D4F8FC0305F023F810BD70B504460D4682
:1024F00000BF94F8B803012801D1022070BD01206B
:1025000084F8B80300BF2946206806F023F900BF0D
:10251000002084F8B80300BF00BFEFE710B5044601
:1025200004F56F71D4F8FC0305F026F810BD10B562
:102530000446206805F064FC206806F049F8002095
:1025400010BD000010B5044600200549087005A024
:1025500006F08EF9D4F8FC0305F057F810BD000022
:102560003101002444657669636520496E207375E6
:102570007370656E64206D6F64652E0D0A00000037
:102580000348006840F0807001490860704700000F
:102590000C48025810B501F067F90949096801F4BF
:1025A00070614FF4807292FAA2F2B2FA82F2D140D4
:1025B000044A515CC840044908600846006810BDE0
:1025C00018440258B09800080000002410B501F02B
:1025D00003F90749096801F07001102292FAA2F28A
:1025E000B2FA82F2D140034A515CC84010BD0000EB
:1025F00020440258B098000870B50146002201201E
:10260000002300249FED811AB0EE410A9FED7F1A4E
:10261000F0EE410A7E4D2D6805F003027C4D2D68D9
:10262000C5F305307A4D2D1D2D6805F01003784D4A
:1026300014352D68C5F3CC0515FB03F501EE105AD2
:10264000B8EE411AB0EE410A22B1012A4DD0022A59
:102650007DD169E06E4D283D2D68C5F340152DB341
:102660006B4D283D2D68C5F3C1066A4D25FA06F469
:10267000B4FBF0F501EE105AF8EE411A9FED661A20
:1026800080EE012A624D10352D68C5F3080501EE74
:10269000105AB8EE411A32EE011AB7EE002A31EEA6
:1026A000021A21EE811AF0EE410A1DE0594DB5FBE8
:1026B000F0F501EE105AF8EE411A9FED571A80EE30
:1026C000012A534D10352D68C5F3080501EE105A47
:1026D000B8EE411A32EE011AB7EE002A31EE021AB4
:1026E00021EE811AF0EE410A5EE04C4DB5FBF0F5AB
:1026F00001EE105AB8EE412A9FED471AC0EE011ABA
:10270000434D10352D68C5F3080501EE105AB8EE9B
:10271000411A31EE811AF7EE001A31EE211A22EE3B
:10272000011AF0EE410A3FE03D4DB5FBF0F501EE38
:10273000105AF8EE411A9FED381A80EE012A344DF6
:1027400010352D68C5F3080501EE105A00E00CE0C5
:10275000B8EE411A32EE011AB7EE002A31EE021A33
:1027600021EE811AF0EE410A1EE02C4DB5FBF0F58A
:1027700001EE105AB8EE412A9FED271AC0EE011A59
:10278000234D10352D68C5F3080501EE105AB8EE3B
:10279000411A31EE811AF7EE001A31EE211A22EEBB
:1027A000011AF0EE410A00BF00BF194D10352D6827
:1027B000C5F346256D1C01EE105AB8EE411AC0EE65
:1027C000811ABCEEE11A81ED001A114D10352D6809
:1027D000C5F306456D1C01EE105AB8EE411AC0EE65
:1027E000811ABCEEE11A81ED011A094D10352D68F0
:1027F000C5F306656D1C01EE105AB8EE411AC0EE25
:10280000811ABCEEE11A81ED021A70BD00000000D1
:10281000284402580090D0030000004600093D0003
:1028200040787D0170B5014600220120002300247C
:102830009FED811AB0EE410A9FED7F1AF0EE410A3A
:102840007E4D2D6805F003027C4D2D68C5F30550C3
:102850007A4D2D1D2D6805F48073784D1C352D683B
:10286000C5F3CC0515FB03F501EE105AB8EE411A7D
:10287000B0EE410A22B1012A4DD0022A7DD169E091
:102880006E4D283D2D68C5F340152DB36B4D283D89
:102890002D68C5F3C1066A4D25FA06F4B4FBF0F5C0
:1028A00001EE105AF8EE411A9FED661A80EE012AE9
:1028B000624D18352D68C5F3080501EE105AB8EEC3
:1028C000411A32EE011AB7EE002A31EE021A21EE59
:1028D000811AF0EE410A1DE0594DB5FBF0F501EE0D
:1028E000105AF8EE411A9FED571A80EE012A534D07
:1028F00018352D68C5F3080501EE105AB8EE411AD7
:1029000032EE011AB7EE002A31EE021A21EE811AD8
:10291000F0EE410A5EE04C4DB5FBF0F501EE105AC9
:10292000B8EE412A9FED471AC0EE011A434D183503
:102930002D68C5F3080501EE105AB8EE411A31EEC4
:10294000811AF7EE001A31EE211A22EE011AF0EE8A
:10295000410A3FE03D4DB5FBF0F501EE105AF8EEAF
:10296000411A9FED381A80EE012A344D18352D6832
:10297000C5F3080501EE105A00E00CE0B8EE411A6C
:1029800032EE011AB7EE002A31EE021A21EE811A58
:10299000F0EE410A1EE02C4DB5FBF0F501EE105AA9
:1029A000B8EE412A9FED271AC0EE011A234D1835C3
:1029B0002D68C5F3080501EE105AB8EE411A31EE44
:1029C000811AF7EE001A31EE211A22EE011AF0EE0A
:1029D000410A00BF00BF194D18352D68C5F34625C3
:1029E0006D1C01EE105AB8EE411AC0EE811ABCEE11
:1029F000E11A81ED001A114D18352D68C5F3064511
:102A00006D1C01EE105AB8EE411AC0EE811ABCEEF0
:102A1000E11A81ED011A094D18352D68C5F30665D7
:102A20006D1C01EE105AB8EE411AC0EE811ABCEED0
:102A3000E11A81ED021A70BD00000000284402581E
:102A40000090D0030000004600093D0040787D0161
:102A50002DE9F041044600250026206800F00060C2
:102A6000B0F1006F30D1606E48B1B0F5801F0DD06D
:102A7000B0F5001F10D0B0F5401F15D113E0F94894
:102A8000006840F40030F74908600FE00221201D83
:102A900002F060FD054609E0022104F1240002F085
:102AA000F1FD054602E001E0012500BF00BF55B978
:102AB000EC482430006820F44010616E0843E94976
:102AC0002431086000E02E43208800F48070B0F5C7
:102AD000807F2DD1606D05281AD2DFE800F0030A4F
:102AE00010171800DF48006840F40030DD49086026
:102AF00010E00021201D02F02DFD05460AE0002116
:102B000004F1240002F0BEFD054603E002E001E00E
:102B1000012500BF00BF55B9D2482430006820F01D
:102B20000700616D0843CF492431086000E02E435F
:102B3000208800F40070B0F5007F33D1A06D8028AC
:102B400017D003DC40B140281CD10CE0C02817D0BE
:102B5000B0F5807F16D114E0C248006840F4003020
:102B6000C049086010E00021201D02F0F3FC05467A
:102B70000AE0002104F1240002F084FD054603E090
:102B800002E001E0012500BF00BF55B9B54824307F
:102B9000006820F4E070A16D0843B2492431086058
:102BA00000E02E43208800F48060B0F5806F38D1BB
:102BB000D4F8A400B0F5800F19D004DC50B1B0F502
:102BC000001F1DD10DE0B0F5C00F17D0B0F5000FFC
:102BD00016D114E0A348006840F40030A149086011
:102BE00010E00021201D02F0B5FC05460AE000219E
:102BF00004F1240002F046FD054603E002E001E096
:102C0000012500BF00BF5DB996482C30006820F454
:102C10006000D4F8A410084392492C31086000E009
:102C20002E43208800F40060B0F5006F38D1D4F84E
:102C3000A800B0F1007F19D004DC50B1B0F1807F62
:102C40001DD10DE0B0F1407F17D0B0F1806F16D1EB
:102C500014E08448006840F400308249086010E0C5
:102C60000021201D02F076FC05460AE0002104F157
:102C7000240002F007FD054603E002E001E0012523
:102C800000BF00BF5DB977482C30006820F0E060DD
:102C9000D4F8A810084373492C31086000E02E4393
:102CA000206800F00070B0F1007F27D1A06CA0B1C7
:102CB000102804D0202809D030280FD10CE0694812
:102CC000006840F400306749086009E00221201DD7
:102CD00002F040FC054603E002E001E0012500BFF0
:102CE00000BF55B95F482030006820F03000A16C6B
:102CF00008435C492031086000E02E43208800F43E
:102D00008050B0F5805F36D1E06DB0F5005F19D02E
:102D100004DC50B1B0F5805F1DD10DE0B0F5405F2F
:102D200017D0B0F5804F16D114E04E48006840F43B
:102D300000304C49086010E00021201D02F00AFC20
:102D400005460AE0002104F1240002F09BFC054640
:102D500003E002E001E0012500BF00BF55B9414892
:102D60002430006820F4E040E16D08433D492431FF
:102D7000086000E02E43208800F40050B0F5005FAA
:102D800034D1206EB0F5403F1DD007DC68B1B0F5FE
:102D9000803F0BD0B0F5003F18D10DE0B0F5802F8B
:102DA00012D0B0F5A02F11D10FE011E00121201DAC
:102DB00002F0D0FB05460BE0012104F1240002F0F3
:102DC00061FC054604E003E002E001E0012500BFEC
:102DD00000BF55B923482430006820F4E020216E5C
:102DE000084320492431086000E02E43208800F485
:102DF0008040B0F5804F38D1D4F8AC00B0F1405FDE
:102E00001DD007DC68B1B0F1805F0BD0B0F1005F7E
:102E100018D10DE0B0F1804F12D0B0F1A04F11D118
:102E20000FE011E00121201D02F094FB05460BE0AC
:102E3000012104F1240002F025FC054604E003E032
:102E400002E001E0012500BF00BF6DB905482C304C
:102E5000006820F0E040D4F8AC10084301492C3160
:102E6000086002E02C4402582E43208800F4004001
:102E7000B0F5004F26D1E06E98B1B0F1805F03D07D
:102E8000B0F1005F0ED106E0FA48006840F400306F
:102E9000F849086008E00121201D02F05BFB0546AF
:102EA00002E001E0012500BF00BF55B9F148243020
:102EB000006820F04050E16E0843EE49243108607C
:102EC00000E02E43206800F08070B0F1807F27D1B1
:102ED000606CA0B1012804D0022809D003280FD1CA
:102EE0000CE0E448006840F40030E249086009E082
:102EF0000221201D02F02EFB054603E002E001E066
:102F0000012500BF00BF55B9DA482030006820F025
:102F10000300616C0843D7492031086000E02E436C
:102F2000206800F48000B0F5800F7DD1D2480068A1
:102F300040F48070D0490860FEF7C6FA074606E004
:102F4000FEF7C2FAC01B642801D9032505E0CA4870
:102F5000006800F480700028F2D000BF8DBBC54827
:102F60004430006800F44070B4F8B01001F44071CF
:102F7000884214D0BF484430006820F44078BD48EF
:102F80004430006840F48030BA4944310860084653
:102F9000006820F4803008600846C0F80080D4F84B
:102FA000B000B0F5807F15D1FEF78EFA074609E034
:102FB000FEF78AFAC01B41F28831884202D9032504
:102FC00007E038E0AB4844300068C0F34000002818
:102FD000EED000BF4DBB00BFB4F8B00000F44070AD
:102FE000B0F5407F0ED1A3481C38006820F47C5116
:102FF000A24AD4F8B000104041EA10109D491C3993
:10300000086007E09B481C38006820F47C50994910
:103010001C390860974844300068B4F8B010C1F318
:103020000B010843934901E006E002E044310860E7
:1030300002E02E4300E02E43207800F0010068B348
:10304000A06F182819D005DC48B1082808D010282E
:1030500016D10BE0202811D0282811D10FE011E063
:103060000121201D02F076FA05460BE0012104F152
:10307000240002F007FB054604E003E002E001E063
:10308000012500BF00BF55B97A482830006820F0FC
:103090003800A16F084377492831086000E02E43CB
:1030A000207800F00200022828D1606F062815D28F
:1030B000DFE800F003040A11121311E00121201DC2
:1030C00002F048FA05460BE0012104F1240002F069
:1030D000D9FA054604E003E002E001E0012500BF63
:1030E00000BF55B963482830006820F00700616FC1
:1030F000084360492831086000E02E43207800F042
:10310000040004282AD1D4F89000062815D2DFE85C
:1031100000F003040A11121311E00121201D02F036
:1031200019FA05460BE0012104F1240002F0AAFA85
:10313000054604E003E002E001E0012500BF00BF16
:103140005DB94C482C30006820F00700D4F890108E
:10315000084348492C31086000E02E43207800F0F5
:103160002000202836D1D4F88C00B0F1405F1DD06B
:1031700007DC68B1B0F1805F0BD0B0F1005F18D10F
:103180000DE0B0F1804F12D0B0F1A04F11D10FE09F
:1031900011E00021201D02F0DDF905460BE00221BF
:1031A00004F1240002F06EFA054604E003E002E0B8
:1031B00001E0012500BF00BF5DB92E48283000683E
:1031C00020F0E040D4F88C1008432A4928310860E8
:1031D00000E02E43207800F04000402836D1D4F89B
:1031E0009800B0F5406F1DD007DC68B1B0F5806F76
:1031F0000BD0B0F5006F18D10DE0B0F5805F12D0A4
:10320000B0F5A05F11D10FE011E00021201D02F008
:10321000A1F905460BE0022104F1240002F032FA84
:10322000054604E003E002E001E0012500BF00BF25
:103230005DB910482C30006820F4E050D4F89810A4
:1032400008430C492C31086000E02E43207800F040
:10325000800080283BD1D4F89C00B0F5C04F24D02A
:103260000EDCA0B1B0F5005F12D0B0F5804F1FD1D9
:1032700014E000002C44025800480258FFFCFF0FE5
:10328000B0F5004F12D0B0F5204F11D10FE011E092
:103290000021201D02F05EF905460BE0022104F139
:1032A000240002F0EFF9054604E003E002E001E04B
:1032B000012500BF00BF4DB9B248006820F460404E
:1032C000D4F89C100843AF49086000E02E432078F2
:1032D00000F00800082816D1D4F88000B0F5805F0F
:1032E00006D1022104F1240002F0CCF906430AE0E1
:1032F000A448001F006820F44050D4F88010084310
:10330000A049091F0860207800F01000102814D18F
:10331000D4F89400B0F5807F06D1022104F1240096
:1033200002F0B0F9064308E09648006820F44070C7
:10333000D4F89410084393490860206800F40020F2
:10334000B0F5002F26D1D4F8A00030B1B0F5803F01
:1033500009D0B0F5003F0ED10CE00021201D02F095
:10336000F9F8054609E0022104F1240002F08AF987
:10337000054602E001E0012500BF00BF4DB98148CC
:10338000006820F44030D4F8A01008437D4908605C
:1033900000E02E43206800F48020B0F5802F2DD16E
:1033A000D4F88400B0F5801F06D0B0F5001F0CD013
:1033B000B0F5401F11D10FE072482C38006840F47E
:1033C000003070492C39086009E0012104F1240023
:1033D00002F058F9054602E001E0012500BF00BFF8
:1033E0005DB96848001F006820F44010D4F88410CC
:1033F00008436449091F086000E02E43206800F478
:103400008030B0F5803F24D1E06C18B1B0F5803F3A
:103410000FD108E05B482C38006840F4003059496F
:103420002C39086007E00221201D02F093F80546C0
:1034300001E0012500BF00BF55B952480C380068B3
:1034400020F48030E16C08434E490C39086000E0FC
:103450002E43206800F00050B0F1005F05D102213A
:1034600004F1240002F00EF90643206800F4003055
:10347000B0F5003F27D1E06FA0B1B0F5807F06D056
:10348000B0F5007F0CD0B0F5407F0CD109E03D488D
:103490002C38006840F400303A492C39086004E0C8
:1034A00003E002E001E0012500BF00BF55B9354847
:1034B000001F006820F44070E16F08433149091F84
:1034C000086000E02E43206800F48010B0F5801FF3
:1034D00009D12C480838006820F00040216F0843CB
:1034E000284908390860206800F08050B0F1805FFA
:1034F0000AD124484838006820F48040D4F8B41039
:103500000843204948390860206800F40010B0F5ED
:10351000001F09D11B480838006820F08070A16E98
:103520000843184908390860206800F08040B0F16D
:10353000804F11D100BF13484838006820F4004084
:1035400010494839086008460068D4F8B8100843A4
:103550000C494839086000BF206800F00040B0F115
:10356000004F09D107480C38006820F04050216D09
:10357000084304490C39086016B90020BDE8F08101
:103580000120FBE75844025870B504460D4600265A
:103590008D48006800F00700A8420ED28A480068F3
:1035A00020F007002843884908600846006800F0BA
:1035B0000700A84201D0012070BD207800F0020071
:1035C000022807D18148006820F00F00E168084315
:1035D0007E490860207800F00100002851D07B4827
:1035E000006820F47060A16808437849086060684A
:1035F000022807D1754818380068C0F34040F8B970
:103600000120D9E76068032807D17048183800689E
:10361000C0F34060A0B90120CEE76068012807D15F
:103620006A4818380068C0F3002048B90120C3E791
:10363000664818380068C0F3800008B90120BBE76D
:1036400062480838006820F00700616808435F4955
:1036500008390860FDF738FF06466068022811D176
:1036600008E0FDF731FF801B41F28831884201D923
:103670000320A1E755480838006800F038001028FA
:10368000EFD13AE06068032811D108E0FDF71CFF94
:10369000801B41F28831884201D903208CE74B48D6
:1036A0000838006800F038001828EFD125E060687D
:1036B000012811D108E0FDF707FF801B41F2883196
:1036C000884201D9032077E740480838006800F0B5
:1036D00038000828EFD110E008E0FDF7F5FE801B68
:1036E00041F28831884201D9032065E7374808381C
:1036F000006800F038000028EFD13348006800F07F
:103700000700A8420ED93048006820F0070028437F
:103710002D4908600846006800F00700A84201D063
:10372000012049E7207800F00400042807D1274849
:10373000006820F07000216908432449086020785F
:1037400000F00800082809D12048001D006820F07A
:103750007000616908431D49091D0860207800F068
:103760001000102809D11948001D006820F4E060FD
:10377000A16908431549091D0860207800F0200060
:10378000202809D111480830006820F07000E16954
:1037900008430E490831086000F066F80B490968D3
:1037A00001F470614FF4807292FAA2F2B2FA82F2DE
:1037B000D140074A515CC840064908600020FDF727
:1037C000A3FE0020F8E60000002000521844025832
:1037D000B09800080000002410B5FEF7DBFE094990
:1037E000096801F00F01012292FAA2F2B2FA82F204
:1037F000D140054A515CC840044908600846006849
:1038000010BD000018440258B098000804000024BD
:1038100010B5FFF7E1FF0749096801F070011022B8
:1038200092FAA2F2B2FA82F2D140034A515CC84045
:1038300010BD00001C440258B098000810B5FFF7F6
:10384000CBFF0749096801F4E0614FF4807292FAF6
:10385000A2F2B2FA82F2D140024A515CC84010BDD5
:103860001C440258B098000870B5012500EE905A2B
:103870000022012100230024DFED861AB0EE610A48
:10388000DFED841AB0EE611A0020834D2D6805F03B
:10389000380535B1082D15D0102D15D0182D7CD137
:1038A00014E07D4D103D2D68C5F3401545B17A4DAE
:1038B000103D2D68C5F3C106784D25FA06F000E0ED
:1038C0007648E5E07648E3E07648E1E0724D183569
:1038D0002D6805F00302704D18352D68C5F30511EC
:1038E0006D4D1C352D6805F001036B4D24352D6899
:1038F000C5F3CC0515FB03F501EE905AF8EE611AFD
:10390000B0EE610A22B1012A4FD0022A7DD16BE0CC
:10391000614D103D2D68C5F340152DB35E4D103D32
:103920002D68C5F3C1065D4D25FA06F4B4FBF1F52B
:1039300001EE905AB8EE612ADFED5B1AC0EE212A43
:10394000554D20352D68C5F3080501EE905AF8EE67
:10395000611A72EEA11AF7EE002A71EEA21A62EE57
:10396000211AB0EE611A1FE04C4DB5FBF1F501EEE6
:10397000905AB8EE612ADFED4C1AC0EE212A464D6E
:1039800020352D68C5F3080501EE905AF8EE611A4E
:1039900072EEA11AF7EE002A00E077E071EEA21AAB
:1039A00062EE211AB0EE611A5EE03D4DB5FBF1F515
:1039B00001EE905AB8EE612ADFED3B1AC0EE212AE3
:1039C000354D20352D68C5F3080501EE905AF8EE07
:1039D000611A72EEA11AF7EE002A71EEA21A62EED7
:1039E000211AB0EE611A3FE02E4DB5FBF1F501EE64
:1039F000905AB8EE612ADFED2C1AC0EE212A264D2E
:103A000020352D68C5F3080500E00EE001EE905A60
:103A1000F8EE611A72EEA11AF7EE002A71EEA21A00
:103A200062EE211AB0EE611A1EE01D4DB5FBF1F5F4
:103A300001EE905AF8EE612ADFED1B1A80EE212A82
:103A4000154D20352D68C5F3080501EE905AF8EEA6
:103A5000611A72EE211AB7EE002A71EE821A62EE36
:103A6000A11AB0EE611A00BF00BF0B4D20352D68C2
:103A7000C5F346256D1C00EE905AF8EE601A81EEF3
:103A8000212AFCEEC21A11EE900A01E0044800BFA0
:103A900000BF70BD00000000104402580090D00329
:103AA00000093D0040787D010000004670B50446E5
:103AB0000025207800F00100002872D0F948006845
:103AC00000F0380010280CD0F648006800F03800EC
:103AD000182812D1F3481830006800F003000228BB
:103AE0000BD1F04810380068C0F3404000286DD07A
:103AF000606800286AD1012070BD00BF6068B0F521
:103B0000803F08D1E7481038006840F48030E5492C
:103B1000103908602EE0606868B9E2481038006823
:103B200020F48030DF49103908600846006820F42E
:103B3000802008601EE06068B0F5A02F0DD1D94844
:103B40001038006840F48020D649103908600846D3
:103B5000006840F4803008600CE0D24810380068FB
:103B600020F48030CF49103908600846006820F4FE
:103B70008020086000BF6068A0B1FDF7A5FC054685
:103B800008E0FDF7A1FC401B41F28831884201D9D1
:103B90000320B1E7C34810380068C0F34040002854
:103BA000EFD013E0FDF790FC054608E0FDF78CFC34
:103BB000401B41F28831884201D903209CE7B94873
:103BC00010380068C0F340400028EFD1207800F0A2
:103BD0000200022847D1B348006800F0380058B10D
:103BE000B048006800F0380018283ED1AD481830C1
:103BF000006800F00300B8BBAA4810380068C0F3A2
:103C0000800018B1E06808B9012075E7A5481038B0
:103C1000006820F01900E1680843A24910390860E3
:103C2000FDF752FC054606E0FDF74EFC401B02285E
:103C300001D9032060E79B4810380068C0F380007A
:103C40000028F1D097480C38006820F47C304FF4FD
:103C50007C3292FAA2F2B2FA82F2216991400843D0
:103C600090490C3908604AE0FFE7E06868B38D4886
:103C70001038006820F01900E168084389491039BC
:103C80000860FDF721FC054606E0FDF71DFC401B22
:103C9000022801D903202FE7824810380068C0F3BA
:103CA00080000028F1D07F480C38006820F47C3078
:103CB0004FF47C3292FAA2F2B2FA82F22169914078
:103CC000084378490C39086019E0764810380068D4
:103CD00020F00100734910390860FDF7F5FB054637
:103CE00006E0FDF7F1FB401B022801D9032003E7A2
:103CF0006C4810380068C0F380000028F1D12078AB
:103D000000F01000102877D16648006800F03800F5
:103D100008280CD06348006800F03800182823D128
:103D200060481830006800F0030001281CD15D488D
:103D300010380068C0F3002020B1E069802801D06D
:103D40000120D9E657480C38006820F0F8404FF0C1
:103D5000F84292FAA2F2B2FA82F2216A9140084342
:103D600050490C39086047E0E06958B34D481038B5
:103D7000006840F080004B4910390860FDF7A4FB53
:103D8000054606E0FDF7A0FB401B022801D90320F1
:103D9000B2E6444810380068C0F300200028F1D093
:103DA00040480C38006820F0F8404FF0F84292FA92
:103DB000A2F2B2FA82F2216A9140084339490C39E1
:103DC000086019E037481038006820F08000354955
:103DD00010390860FDF778FB054606E0FDF774FB37
:103DE000401B022801D9032086E62E4810380068BF
:103DF000C0F300200028F1D1207800F00800082846
:103E000036D16069D0B127486430006840F00100C5
:103E1000244964310860FDF757FB054606E0FDF7CD
:103E200053FB401B022801D9032065E61D4864307E
:103E30000068C0F340000028F1D019E01948643050
:103E4000006820F00100174964310860FDF73CFB71
:103E5000054606E0FDF738FB401B022801D9032088
:103E60004AE6104864300068C0F340000028F1D1F1
:103E7000207800F02000202834D1A069D8B109486A
:103E80001038006840F48050064910390860FDF78A
:103E90001BFB054608E0FDF717FB401B022803D972
:103EA000032029E610440258AF480068C0F34030B0
:103EB0000028F0D016E0AC48006820F48050AA49F1
:103EC0000860FDF701FB054606E0FDF7FDFA401B23
:103ED000022801D903200FE6A3480068C0F3403050
:103EE0000028F2D1207800F0040004287DD19F48FA
:103EF000006840F480709D490860FDF7E5FA0546CA
:103F000006E0FDF7E1FA401B642801D90320F3E540
:103F10009648006800F480700028F2D000BFA068C6
:103F2000012808D190487030006840F001008E49A7
:103F3000703108602DE0A06868B98B487030006867
:103F400020F001008849703108600846006820F0C0
:103F5000040008601DE0A06805280DD1824870307B
:103F6000006840F00400804970310860084600682D
:103F700040F0010008600CE07B487030006820F0E1
:103F800001007949703108600846006820F004009B
:103F9000086000BFA068A0B1FDF796FA054608E0EA
:103FA000FDF792FA401B41F28831884201D9032083
:103FB000A2E56D4870300068C0F340000028EFD0E3
:103FC00013E0FDF781FA054608E0FDF77DFA401B96
:103FD00041F28831884201D903208DE56248703072
:103FE0000068C0F340000028EFD1606A00287CD050
:103FF0005D481030006800F03800182876D0606AFC
:10400000022874D15848006820F080705649086032
:10401000FDF75AFA054606E0FDF756FA401B02285E
:1040200001D9032068E550480068C0F340600028CB
:10403000F2D100BFD4E90A1041EA00104A49283100
:10404000096840F2F3329143084347492831086038
:10405000208E401EC0F30800616B491E4FF47E4263
:1040600002EA41210843218F491ED20102EA01419F
:1040700008433C21095D491E120202EA016108431E
:1040800039493031086000BF081D00684FF6F871EB
:1040900088434FF6F87292FAA2F2B2FA82F2A16C59
:1040A000914008433049343108602F482C30006873
:1040B00020F00C00216C08432B492C310860084685
:1040C000006820F00200616C084327492C31086029
:1040D0000846006840F4803008600846006840F4F4
:1040E000003008600846006802E03BE038E01FE06E
:1040F00040F4802008600846006840F00100086035
:104100001948006840F0807017490860FDF7DCF935
:10411000054606E0FDF7D8F9401B022801D9032027
:10412000EAE411480068C0F340600028F2D019E0CA
:104130000D48006820F080700B490860FDF7C4F955
:10414000054606E0FDF7C0F9401B022801D903200F
:10415000D2E405480068C0F340600028F2D101E0D5
:104160000120C9E40020C7E4004402580048025876
:1041700070B50446002500260CB9012070BD606AA8
:1041800000B900BFA06AB0F5800F00D100BF8E4912
:10419000206888420CD08D492068884208D08C491C
:1041A0002068884204D0E0680F2801D90120E5E7A3
:1041B000204601F095FC064683492068884209D0D4
:1041C00082492068884205D081492068884201D010
:1041D000082E0DD87C492068884207D07B4920688A
:1041E000884203D07A492068884203D1102E01D931
:1041F0000120C3E7A06AB0F5800F1DD17249206885
:1042000088420DD071492068884209D070492068E1
:10421000884205D0206BB0F5702F01D90120ADE7A1
:10422000206B10B9A089050400E0256BE068B0EBB5
:10423000154F01D90120A1E794F8810028B9002089
:1042400084F88000204600F0C5F8022084F8810040
:104250002068006820F0010021680860A069B0F1C2
:10426000806F0BD16068B0F5800F07D1A06B28B9C3
:104270002068006840F4805021680860A16AE06905
:1042800008432843E16B0843E168084321688860DC
:10429000616A606B0843A16B0843A1690843216907
:1042A000084361690843216A084361680843E16C77
:1042B0000843A1680843A16C0843A16D0843216825
:1042C000C860A06AB0F5800F4DD1206C012806D1DE
:1042D0002068006840F400402168086005E020681C
:1042E000006820F4004021680860606C012806D155
:1042F0002068006840F480402168086005E020687C
:10430000006820F48040216808602F4920688842B6
:104310000AD02E492068884206D02D49206888425C
:1043200002D0B5F5702F0ED027492068884207D0FB
:1043300026492068884203D025492068884209D14F
:10434000B5F5F81F06D12068006840F400502168D8
:10435000086005E02068006820F4005021680860CB
:104360002168E06A0864606888B9A06A38B9206882
:10437000806820F4C05040F40060216888602068A4
:10438000806820F4C06040F4806021688860206804
:10439000006D20F0010021680865606800F480006D
:1043A000B0F5800F07D12068C06820F00040616D33
:1043B00008432168C8600020C4F88400012084F804
:1043C00081000020DAE600000030014000380040A3
:1043D000003C004010B5B6B0044600BF1A48006863
:1043E00040F00200184908600846006800F002002A
:1043F000019000BF00BF00BF13480830006840F4C0
:1044000080401149083108600846006800F4804087
:10441000019000BF00BF4FF480500290002019901F
:1044200002A8FEF715FB4FF4604031900220329055
:1044300001203390032034900520359031A90348A2
:10444000FCF712FF36B010BDE044025800040258D9
:104450002DE9F84F0446884691461D460A9E0027DE
:10446000BA4600BF94F88000012802D10220BDE8BE
:10447000F88F012084F8800000BFFDF725F807467B
:1044800094F88100012812D06068B0F5800F05D142
:10449000A06818B994F88100042808D04FF0020AE7
:1044A00000BF002084F8800000BF5046DFE7B8F16D
:1044B000000F03D0B9F1000F00D045B94FF0010A49
:1044C00000BF002084F8800000BF5046CFE794F87A
:1044D0008100042802D0052084F881000020C4F85F
:1044E0008400C4F86490A4F86A50A4F86850C4F832
:1044F0005C80A4F86250A4F8605020676067206870
:1045000040686FF30F002843216848602068006806
:1045100040F00100216808606068B0F5800F05D1A7
:104520002068006840F4007021680860E0680F2887
:104530004CD942E0B4F8620088B12068406900F0CC
:10454000020002280BD1E06D006821680862E06D6E
:10455000001DE065B4F86200401EA4F86200B4F8E3
:104560006A0088B12068406948F20801084058B1E3
:104570002068006B616E0860606E001D6066B4F8B4
:104580006A00401EA4F86A00701CB0B1FCF79CFFE2
:10459000C01BB04211D3204601F024FA00BF002016
:1045A00084F8800000BFD4F8840040F48070C4F820
:1045B0008400012084F8810059E7B4F862000028E3
:1045C000B8D1B4F86A000028B4D10FE1E068072838
:1045D00071D966E0B4F8620020B32068406900F049
:1045E000020002281ED1B4F8620001280ED9E06B47
:1045F00060B1E06D006821680862E06D001DE06553
:10460000B4F86200801EA4F862000BE0E06D008840
:1046100021680884E06D801CE065B4F86200401EEB
:10462000A4F86200B4F86A0010B32068406900F48E
:104630006040E8B12068406900F4004060B1206843
:10464000006B616E0860606E001D6066B4F86A0001
:10465000801EA4F86A000BE02068008E616E08805E
:10466000606E801C6066B4F86A00401EA4F86A00A0
:10467000701CB0B1FCF728FFC01BB04211D320461C
:1046800001F0B0F900BF002084F8800000BFD4F82A
:10469000840040F48070C4F88400012084F8810014
:1046A000E5E6B4F86200002894D1B4F86A00002866
:1046B00090D19BE0FFE790E0B4F8620058B3206827
:1046C000406900F00200022833D1B4F862000328E8
:1046D0000FD9E06B40280CD9E06D006821680862B2
:1046E000E06D001DE065B4F86200001FA4F86200F0
:1046F0001FE0B4F8620001280ED9E06B60B1E06DF4
:10470000008821680884E06D801CE065B4F86200D0
:10471000801EA4F862000CE0E06D0078216881F84A
:104720002000E06D401CE065B4F86200401EA4F873
:104730006200B4F86A0048B32068406900F4604041
:1047400020B32068406900F4004060B12068006B2D
:10475000616E0860606E001D6066B4F86A00001F3C
:10476000A4F86A0020E02068406900F4C040B0F579
:10477000005F0CD92068008E616E0880606E801C1E
:104780006066B4F86A00801EA4F86A000CE0206835
:1047900090F83000616E0870606E401C6066B4F87E
:1047A0006A00401EA4F86A00701CB0B1FCF78CFED1
:1047B000C01BB04211D3204601F014F900BF002005
:1047C00084F8800000BFD4F8840040F48070C4F8FE
:1047D0008400012084F8810049E6B4F862000028D2
:1047E0007FF46AAFB4F86A000028F9D13B46002292
:1047F00008212046009601F080F928B1D4F8840001
:1048000040F02000C4F88400204601F0EBF800BF1F
:10481000002084F8800000BF012084F88100D4F8D3
:10482000840008B1012022E6002020E6042808D1F7
:104830004FF0E021096941F004014FF0E0221161DD
:1048400007E04FF0E021096921F004014FF0E02278
:104850001161704770B504462546681EB0F1807F2F
:1048600001D301200FE0681E4FF0E02148610F21C5
:104870004FF0FF3004F026F800204FF0E02188616F
:1048800007200861002070BD704770470146002274
:10489000002391F8792091F87A3042EA03007047BA
:1048A0002DE9F04104462068C56920680768206842
:1048B000866805F00F08B8F1000F0DD105F0200053
:1048C00050B107F0200010B906F0805020B120460A
:1048D00001F0A5FBBDE8F081B8F1000F72D05D4892
:1048E000304018B907F4907000287AD005F0010024
:1048F00048B107F4807030B1012021680862E06F90
:1049000040F00100E06705F0020048B106F0010048
:1049100030B1022021680862E06F40F00400E067D7
:1049200005F0040048B106F0010030B10420216810
:104930000862E06F40F00200E06705F0080078B11F
:1049400007F0200028B906F0805010B906F00100E9
:1049500030B1082021680862E06F40F00800E0678D
:10496000E06F70B305F0200040B107F0200010B9EF
:1049700006F0805010B1204601F051FBE06F00F0CE
:10498000080020B92068806800F0400018B3204675
:1049900001F025FB2068806800F04000B8B1206875
:1049A000806820F0400021688860606F58B12A4814
:1049B000616F0865606FFCF7BDFB10B1606F016D42
:1049C00088470DE00DE02046FFF75FFF08E0204636
:1049D000FFF75BFF04E02046FFF757FF0020E0678A
:1049E00078E705F4801078B106F4800060B14FF4E8
:1049F000801021680862202084F8790084F87A0009
:104A00002046FFF741FF65E705F0800048B107F059
:104A1000800010B906F4000018B1204602F016F824
:104A200058E705F0400030B107F0400018B12046CB
:104A300001F0E5FA4EE705F4000040B107F08040D0
:104A400028B12068006820F080402168086000BF1D
:104A500040E7000001000010C75F000810B50446E1
:104A60000CB9012010BDA06900B100E000BF94F8AE
:104A7000790028B9002084F87800204600F02AF850
:104A8000242084F879002068006820F00100216863
:104A90000860204601F008FB012800D1E2E7606BC6
:104AA00010B1204601F0E0F92068406820F4904001
:104AB000216848602068806820F02A0021688860AA
:104AC0002068006840F0010021680860204601F07D
:104AD00040FAC7E710B586B00446214920688842ED
:104AE0003BD100BF1F48006840F001001D4908602D
:104AF0000846006800F00100009000BF00BF00BF42
:104B000018481030006840F0100016491031086055
:104B10000846006800F01000009000BF00BF4FF48E
:104B20000070019002200290012003900220049066
:104B30000720059001A90C48FCF796FB4FF4806014
:104B4000019001A90848FCF78FFB2520FCF767FDC1
:104B5000032211462520FCF772FD06B010BD0000AF
:104B600000100140E04402580000025810B503460E
:104B700093F87A00202867D101B10AB9012010BD4D
:104B800000BF93F87800012801D10220F7E7012047
:104B900083F8780000BF5966A3F86820A3F86A205C
:104BA00000BF9868B0F5805F0AD1186920B940F25B
:104BB000FF10A3F86C001CE0FF20A3F86C0018E0C5
:104BC000986848B9186918B9FF20A3F86C0010E07C
:104BD0007F20A3F86C000CE09868B0F1805F08D1EA
:104BE000186918B97F20A3F86C0002E03F20A3F8F1
:104BF0006C0000BF0020D867222083F87A0000BF35
:104C0000002083F8780000BF1868806840F0010039
:104C10001C68A0601868006800F0005060B1186857
:104C2000006840F480701C6820601868806840F05C
:104C300080501C68A06005E01868006840F490701F
:104C40001C68206000209AE7022098E71D4A01684E
:104C5000914236D11C49098801F4004189BB1A49A7
:104C6000098801F4804171B1184909780A2903D0F3
:104C70000021154A118024E01349098841F40041BC
:104C8000114A11801DE0114909780D2906D10E49FC
:104C9000098841F480410C4A118012E00B490978DF
:104CA000094A1288C2F30D02094B99540649098832
:104CB000491C054A118011460988C72901DD0021D8
:104CC00011807047001001401000002412000024E1
:104CD0000C040024704700BFFEE730B50B460021EE
:104CE00000BF16E00A24B4EB107F05D9302404EB92
:104CF000107403F8114005E0412404EB10740A3CE1
:104D000003F81140000100254C00641C1D554C1C8B
:104D1000E1B29142E6DB30BD00B587B000BF1A4872
:104D2000006840F00400184908600846006800F078
:104D30000400019000BF00BF00BF0846006840F0BB
:104D4000100008600846006800F01000019000BFE5
:104D500000BF08200290002003900120049003204F
:104D6000059002A90948FCF77FFA20200290002054
:104D70000390012004900320059002A90448FCF749
:104D800073FA07B000BD0000E0440258001002585A
:104D90000008025870B5054600240E484388028872
:104DA0000021084600F0F0F90A48008809494988BE
:104DB00000FB01F60021084600F0D2F900F0EEFAFF
:104DC00000BF03E0284600F09DFA641CB442F9D30A
:104DD00070BD0000404D042470B505467DB900202B
:104DE0002F498871F02008804FF4A07048802C2053
:104DF00008812A2048812B208881002444E0012D4D
:104E00000FD10020264988714FF4A0700880F0204F
:104E100048802C2008812A2048812B208881012469
:104E200032E0022D0FD101201D498871F020088049
:104E30004FF4A07048802C2008812A2048812B2024
:104E40008881022420E0032D0FD1012014498871AC
:104E50004FF4A0700880F02048802C2008812A2080
:104E600048812B20888103240EE000200C498871A2
:104E7000F02008804FF4A07048802C2008812A2060
:104E800048812B208881002405484388028800211E
:104E9000084600F079F9204600F046F970BD0000A0
:104EA000404D042470B506460C4615460A4948890B
:104EB00000F05CFA304600F025FA0749888900F0D6
:104EC00055FA204600F01EFA0349088900F04EFA10
:104ED000284600F017FA70BD404D042400B587B095
:104EE00000BF1B48006840F00200194908600846EE
:104EF000006800F00200019000BF00BF41F2030013
:104F000002900120039004900320059002A911480B
:104F1000FCF7AAF9012211460E48FCF7CFFA01224C
:104F200002210C48FCF7CAFA012211030948FCF7D8
:104F3000C5FA00F0F1FC4FF0805000F031FD00F0B8
:104F40000BF8012211460348FCF7B8FA07B000BD80
:104F5000E04402580004025810B500224FF480418A
:104F60000748FCF7ABFA322004F0E2F90122910382
:104F70000348FCF7A3FA1E2004F0DAF910BD000084
:104F80000004025810B5FFF7A9FF00F0B3F9322072
:104F900004F0CEF9362000F0E9F9002000F0CEF957
:104FA0003A2000F0E3F9052000F0C8F9B22000F043
:104FB000DDF90C2000F0C2F90C2000F0BFF9002050
:104FC00000F0BCF9332000F0B9F9332000F0B6F955
:104FD000B72000F0CBF9352000F0B0F9BB2000F08D
:104FE000C5F9192000F0AAF9C02000F0BFF92C2063
:104FF00000F0A4F9C22000F0B9F9012000F09EF9F8
:10500000C32000F0B3F9122000F098F9C42000F09A
:10501000ADF9202000F092F9C62000F0A7F90F208A
:1050200000F08CF9D02000F0A1F9A42000F086F95E
:10503000A12000F083F9E02000F098F9D02000F0E2
:105040007DF9042000F07AF90D2000F077F91120A5
:1050500000F074F9132000F071F92B2000F06EF9C4
:105060003F2000F06BF9542000F068F94C2000F06C
:1050700065F9182000F062F90D2000F05FF90B20AF
:1050800000F05CF91F2000F059F9232000F056F9D8
:10509000E12000F06BF9D02000F050F9042000F07E
:1050A0004DF90C2000F04AF9112000F047F91320C7
:1050B00000F044F92C2000F041F93F2000F03EF9C7
:1050C000442000F03BF9512000F038F92F2000F087
:1050D00035F91F2000F032F91F2000F02FF92020B1
:1050E00000F02CF9232000F029F9212000F03EF9EE
:1050F000112000F03BF9782004F01AF9292000F083
:1051000035F9C82004F014F90020FFF765FE0122EC
:1051100011460448FCF7D2F94FF6FF70FFF73AFE4C
:1051200010BD00000004025870B50546002435B1DA
:10513000012D06D0022D07D0032D0BD107E000BFB3
:1051400008E044F0600405E044F0C00402E044F0EC
:10515000A00400BF00BF2146362000F027F970BD33
:1051600070B505460C460749488900F0FFF8284607
:1051700000F0C8F80349888900F0F8F8204600F0EC
:10518000C1F870BD404D04242DE9F04107460C469E
:1051900015461E467819401E85B2A019401E86B2DB
:1051A0000A49488900F0E2F8384600F0ABF8284692
:1051B00000F0A8F80549888900F0D8F8204600F0EA
:1051C000A1F8304600F09EF8BDE8F081404D04247F
:1051D0002DE9F84F80460E4617461C46B34620463A
:1051E000E31704EB5373DB1021464FEAE47C04EB36
:1051F0005C7C4FEAEC0CA4EBCC0CBCF1000F02D0B1
:105200004FF0010C01E04FF0000C6344224604EB28
:10521000D27C4FEA6C0C03FB0CF3DBB20093A7F1DA
:105220002000C7B2002555E00C2C07D107EB470042
:105230002B4901EB800010F8059013E0102C05D1EC
:10524000284800EB071010F805900BE0182C07D148
:1052500007EBC700244901EB800010F8059001E03E
:10526000BDE8F88F4FF0000A2EE009F0800028B169
:10527000314640460A9AFFF715FE07E00B9828B919
:105280001A48028831464046FFF70CFE4FEA496053
:105290004FEA1069701C86B215484088B04200DCA5
:1052A000DEE7A6EB0B00A0420AD15E4608F1010042
:1052B0001FFA80F80E480088404500DCD0E706E081
:1052C0000AF1010000F0FF0ABAF1080FCDDB00BFC0
:1052D000681CC5B200988542A6DB00BFC0E700008D
:1052E00038990008AC9D00089CA30008E201002446
:1052F000404D042410B5012000F038F8322004F0AD
:1053000017F810BD10B5044600224FF480510A482A
:10531000FCF7D4F8012202210748FCF7CFF820124D
:1053200000F02EFBE0B200F02BFB0122110302483B
:10533000FCF7C4F810BD00000004025810B5044684
:1053400000224FF480510848FCF7B8F801220221EE
:105350000548FCF7B3F8204600F012FB01221103C8
:105360000148FCF7ABF810BD0004025810B5044624
:1053700000224FF480510848FCF7A0F800220221D7
:105380000548FCF79BF8E0B200F0FAFA012211039D
:105390000148FCF793F810BD0004025810B502490B
:1053A0000889FFF7E3FF10BD404D042470B50546A2
:1053B0000C462846FFF7DAFFE0B2FFF7BFFF70BDEB
:1053C00000B587B000BF0F48006840F001000D49EC
:1053D00008600846006800F00100019000BF00BFAF
:1053E000022002900120039004900320059002A95E
:1053F0000548FBF739FF012202210348FCF75EF85C
:1054000007B000BDE0440258000002580EB500206D
:105410000121009103230A46CDE90110122148061B
:1054200000F001F80EBD2DE9FF4704460D46164673
:105430001F46DDE90D9ADDF83080FCF7B9F8012050
:105440008DF80000F0B28DF801000194E8B28DF8FB
:10545000080000208DF809008DF80A008DF80B7007
:105460008DF80C008DF80D808DF80E908DF80FA042
:105470006846FCF76FF80420FCF7B0F8002004B091
:10548000BDE8F08700BFFEE77047000010B5024896
:10549000FCF71CFB10BD0000DC0500242DE9F84FD3
:1054A00007460E46D7F8008000240025A146A246F4
:1054B000C6EBC60107F1380000EB8104D4E9050111
:1054C000451AA068A84200D2A568E81CC11700EBE5
:1054D00091714FEAA1091AE0D4E90501451AA068C3
:1054E000A84200D2A568E81CC11700EB91714FEAF1
:1054F000A109387CABB2F2B200904046E16803F0FB
:1055000043F9E0682844E060A0692844A06108F5F8
:10551000106000EB4610806980B2484506D9D4E996
:105520000510884202D260690028D5D1002D0CDC1C
:10553000012000FA06FA40F6340050F8080020EA8C
:105540000A0040F6340141F808000020BDE8F88F59
:10555000704700002DE9F04104460E4600274848F8
:10556000006800F00300032802D10120BDE8F081AB
:1055700043482838006820F0806041492839086095
:10558000FBF7A2FF054606E0FBF79EFF401B022843
:1055900001D90320EAE73A4828380068C0F3C06020
:1055A0000028F1D100BF3648006820F47C30216823
:1055B00040EA013032490860A088401EC0F308006C
:1055C000A168491E4FF47E4202EA41210843A189A5
:1055D000491ED20102EA01410843217C491E120200
:1055E00002EA0161084326491031086000BF2448DF
:1055F000001D006820F0C000616908432049091DB2
:1056000008600846006820F02000A16908431C4992
:10561000091D08602EB90846006840F400200860A3
:1056200012E0012E08D11648001D006840F48010D9
:105630001349091D086007E01148001D006840F487
:1056400000100F49091D08600D482838006840F017
:1056500080600B4928390860FBF736FF054606E0F5
:10566000FBF732FF401B022801D903207EE70448E4
:1056700028380068C0F3C0600028F1D0384675E7CC
:10568000284402582DE9F04104460E4600274848B8
:10569000006800F00300032802D10120BDE8F0817A
:1056A00043482838006820F0805041492839086074
:1056B000FBF70AFF054606E0FBF706FF401B022842
:1056C00001D90320EAE73A4828380068C0F340705F
:1056D0000028F1D100BF3648006820F07C70218896
:1056E00040EA015032490860A088401EC0F308001B
:1056F000A168491E4FF47E4202EA41210843A18974
:10570000491ED20102EA01410843217C491E1202CE
:1057100002EA0161084326491831086000BF2448A5
:10572000001D006820F44060616908432049091D9C
:1057300008600846006820F40070A16908431C490D
:10574000091D08602EB90846006840F48000086012
:1057500012E0012E08D11648001D006840F4000038
:105760001349091D086007E01148001D006840F05A
:1057700080700F49091D08600D482838006840F006
:1057800080500B4928390860FBF79EFE054606E06D
:10579000FBF79AFE401B022801D903207EE704484C
:1057A00028380068C0F340700028F1D0384675E70B
:1057B0002844025830B50A460446202300BF00BFE3
:1057C00000BFBFF34F8F00BF00BF00BF03E00B4D12
:1057D0002C601C44D21A002AF9DC00BF00BF00BFB5
:1057E000BFF34F8F00BF00BF00BF00BF00BF00BFAF
:1057F000BFF36F8F00BF00BF00BF30BD68EF00E098
:1058000010B50023234C236000BF00BF00BFBFF3CF
:105810004F8F00BF00BF00BF231F1868C0F34E3179
:1058200000BFC0F3C90200BF43F6E07303EA4113AF
:105830004FF0404404EA82742343174C236000BFB6
:1058400000BF131EA2F10102EED10B1EA1F1010156
:10585000E7D100BF00BF00BFBFF34F8F00BF00BF45
:1058600000BF0C4B703B1B6843F48033094C703C09
:10587000236000BF00BF00BFBFF34F8F00BF00BF5A
:1058800000BF00BF00BF00BFBFF36F8F00BF00BFEE
:1058900000BF10BD84ED00E060EF00E000BF00BF7E
:1058A00000BFBFF34F8F00BF00BF00BF00BF00BFEE
:1058B00000BFBFF36F8F00BF00BF00BF00201449BF
:1058C000086000BF00BF00BFBFF34F8F00BF00BF25
:1058D00000BF00BF00BF00BFBFF36F8F00BF00BF9E
:1058E00000BF0C48006840F400300A49086000BF5F
:1058F00000BF00BFBFF34F8F00BF00BF00BF00BF9E
:1059000000BF00BFBFF36F8F00BF00BF00BF704775
:1059100050EF00E014ED00E010B51748174908609B
:105920004FF4800048600021144881600721C16065
:105930004FF00071016149104161890081610021CE
:1059400041634FF0004141654FF0E041C1610021EA
:105950000162416281620721C162FEF709FC0748CA
:105960000068006840F00100044909680860FF20F1
:1059700000F006F810BD0000003800405405002477
:1059800001B582B04FF47A70012301AA02A90090F8
:105990000248FEF75DFD9DF804000EBD540500248D
:1059A0000F490968096821F001010D4A1268116068
:1059B0000B490968896821F0E041094A1268916041
:1059C0000749096889680143054A126891600449DA
:1059D0000968096841F00101014A126811607047C5
:1059E00054050024026851690268926942F0080275
:1059F00003689A610268926942F0100203689A6132
:105A00000268126822F0010203681A6002681269D3
:105A100040F26B339A4303681A610268926822F479
:105A2000404203689A6090F88120042A0ED001F069
:105A300020025AB1D0F8842042F08002C0F88420BD
:105A40000268926942F0200203689A6190F881200E
:105A5000032A21D001F040025AB1D0F8842042F04C
:105A60000402C0F884200268926942F04002036890
:105A70009A61826AB2F5800F0ED101F080025AB1AC
:105A8000D0F8842042F00202C0F8842002689269B3
:105A900042F0800203689A6101F400725AB1D0F8B2
:105AA000842042F00102C0F884200268926942F426
:105AB000007203689A6101F480725AB1D0F88420B0
:105AC00042F00802C0F884200268926942F48072B1
:105AD00003689A610022A0F86220A0F86A2070474B
:105AE00010B501460124C86B04EB5013C868421C72
:105AF000D01DC20802FB03F010BD2DE9F04106469F
:105B00000C4617469846069D0BE0681C48B12DB11F
:105B1000FBF7DAFCA0EB0800A84202D90320BDE89D
:105B2000F081306840692040A04201D1012000E0AE
:105B30000020B842E9D00020F1E770472DE9F04F8E
:105B400093B00546884691461C46AB462046E21770
:105B500004EB5272D2102146E31704EB5373DB10AF
:105B6000A4EBC3030BB1012300E000231A446243FA
:105B7000D7B20C2C06D0102C04D0182C02D013B0A5
:105B8000BDE8F08F23463A4669464846FBF782FA5D
:105B900000262FE01DF8060012904FF0000A24E0C6
:105BA000129800F0800028B1414628461C9AFFF761
:105BB00079F907E01D9828B910480288414628461F
:105BC000FFF770F912984006000E1290681C85B21B
:105BD000A5EB0B00A04204D15D4608F101001FFABD
:105BE00080F80AF1010000F0FF0ABAF1080FD7DBD4
:105BF000701CC6B2BE42CDDB00BFC0E7E20100248C
:105C00002DE9FF5F07460E4691469A46DDE90F4BA8
:105C10000E9DB8460396002002904EE0029878BB95
:105C20002878802802DD0120029046E004EBD47140
:105C300008EB0902A2EB6101B94202DA301986B21F
:105C4000474603985044001BB04200DA38E02878F9
:105C50000D2804D1301986B247466D1C08E0119812
:105C6000CDE900B02A78234631463846FFF7B0FA2E
:105C70006D1C204604EBD07107EB61018FB21CE074
:105C8000FFE70020029008EB0900001BB84202DA8F
:105C9000301986B2474603985044001BB04200DAE0
:105CA0000EE0119823462A463146CDE900B0384629
:105CB000FFF744FFAD1C381987B228780028ADD112
:105CC00000BFBDE8FF9F00002DE9F0419CB0804679
:105CD0000C4615461E4600273A48006820F004008E
:105CE0003849086000BF0020009036480C3000683A
:105CF00040F4404033490C3108600846006800F425
:105D00004040009000BF00BF00BF2E480C3000682C
:105D100000F40050B0F5005FF7D1212001904FF45E
:105D2000803002900120079000200490089002200B
:105D30000A9002210B91CDF834800C940E950F96A9
:105D400000211291082111910021139101A8FDF762
:105D5000ADFE07460FB100BFFEE73F2014900320C1
:105D600015900020169008201790402019900001EF
:105D70001A904020189050201B90022114A8FDF783
:105D800003FC07460FB100BFFEE70F48006840F074
:105D900080000D49086000BF0B48F430006840F0F7
:105DA00002000949F43108600846006800F002006A
:105DB000009000BF00BFFBF74DFA00201CB0BDE80B
:105DC000F08100000C4802580044025810B5FBF75F
:105DD00081FB10BD2048006840F470001E49086037
:105DE0001E48006840F001001C49086000201B4963
:105DF00010310860194800681949084017490860BF
:105E00000020164918310860091D0860091D086046
:105E1000124928310860091D0860091D0860091D24
:105E20000860091D0860091D0860091D0860091D3A
:105E300008600A48006820F48020084908600020B3
:105E4000064960310860012006490860C006024921
:105E5000803908607047000088ED00E00044025877
:105E60007FEDF6EA0881005190F8341001F001014D
:105E700039B10168496821F40031826B114302682D
:105E8000516090F8341001F0020139B1016849689D
:105E900021F48031C26B11430268516090F83410D4
:105EA00001F0040139B10168496821F48021026CD4
:105EB00011430268516090F8341001F0080139B1C3
:105EC0000168496821F40041426C11430268516045
:105ED00090F8341001F0100139B10168896821F49B
:105EE0008051826C11430268916090F8341001F087
:105EF000200139B10168896821F40051C26C114355
:105F00000268916090F8341001F0400199B1016885
:105F1000496821F48011026D114302685160016DDE
:105F2000B1F5801F07D10168496821F4C001426DB5
:105F300011430268516090F8341001F0800139B1CA
:105F40000168496821F40021826D114302685160A3
:105F5000704738B5044600250020E067FBF7B4FA27
:105F600005462068006800F0080008280CD16FF092
:105F70007E402B4600224FF400110090204600F096
:105F8000A6FD08B1032038BD2068006800F00400B9
:105F900004280CD16FF07E402B4600224FF4800184
:105FA0000090204600F093FD08B10320EBE720208D
:105FB00084F8790084F87A0000BF002084F8780023
:105FC00000BF00BFDFE770B50546AC6B0020A4F84A
:105FD0006A00A4F862002046FEF757FC70BD016815
:105FE000096821F49071026811600168896821F0E4
:105FF000010102689160202180F87A10704710B585
:1060000004462068006820F04000216808602020D5
:1060100084F879002046FEF75DFE002010BD2DE9D2
:10602000F0410446B4F86C7094F87A00222833D119
:106030002068858CA068B0F5805F09D1206938B9E7
:10604000666E05EA07003080606E801C606605E0C1
:10605000F8B22840626E511C61661070B4F86A0094
:10606000401E80B2A4F86A00A0B92068006820F43D
:106070009070216808602068806820F00100216825
:106080008860202084F87A002046FEF7DFFD00209B
:10609000BDE8F0810020FBE72068008B40F008009D
:1060A000216808830220F3E72DE9F04F89B0044608
:1060B00000254FF08008A946AA4600200890FA491A
:1060C0002068884201D1012000E0002000B100E0FA
:1060D00000BFA06AB0F1005F00D100BF2169A068D5
:1060E000084361690843E16940EA0105A06A054384
:1060F00020680068ED49084028432168086020684E
:10610000406820F44050E168084321684860A56970
:10611000E5492068884201D1012000E0002008B94B
:10612000206A0543A06AB0F1005F03D1D4E90B01F6
:106130000843054320688068DD49084028432168FA
:1061400088602068C06A20F00F00616A08432168F7
:10615000C86200BFD7492068884224D1D648006869
:1061600000F03800182814D005DC48B108280AD0FF
:10617000102817D10AE020280ED0282812D10EE0CE
:106180004FF001080EE04FF004080BE04FF040081C
:1061900008E04FF0080805E04FF0100802E04FF06B
:1061A000200800BF17E1C549206888421DD1C248B8
:1061B000006800F00700062816D2DFE800F00306AA
:1061C000090C0F124FF000080EE04FF004080BE02E
:1061D0004FF0400808E04FF0080805E04FF01008C5
:1061E00002E04FF0200800BFF5E0B5492068884282
:1061F0001DD1B148006800F00700062816D2DFE87C
:1062000000F00306090C0F124FF000080EE04FF0EB
:1062100004080BE04FF0400808E04FF0080805E0E4
:106220004FF0100802E04FF0200800BFD3E0A5496E
:10623000206888421DD1A048006800F007000628A9
:1062400016D2DFE800F00306090C0F124FF0000829
:106250000EE04FF004080BE04FF0400808E04FF06C
:10626000080805E04FF0100802E04FF0200800BFDA
:10627000B1E09549206888421DD18F48006800F040
:106280000700062816D2DFE800F00306090C0F12FB
:106290004FF000080EE04FF004080BE04FF040080C
:1062A00008E04FF0080805E04FF0100802E04FF05A
:1062B000200800BF8FE085492068884224D17E48AD
:1062C000006800F03800182814D005DC48B1082810
:1062D0000AD0102817D10AE020280ED0282812D181
:1062E0000EE04FF001080EE04FF004080BE04FF015
:1062F000400808E04FF0080805E04FF0100802E001
:106300004FF0200800BF66E07149206888421DD127
:106310006948006800F00700062816D2DFE800F0A0
:106320000306090C0F124FF000080EE04FF00408AE
:106330000BE04FF0400808E04FF0080805E04FF090
:10634000100802E04FF0200800BF44E061492068D7
:1063500088421DD15848006800F00700062816D270
:10636000DFE800F00306090C0F124FF000080EE002
:106370004FF004080BE04FF0400808E04FF0080829
:1063800005E04FF0100802E04FF0200800BF22E0C7
:106390004549206888421ED14748001D006800F02A
:1063A0000700062816D2DFE800F00306090C0F12DA
:1063B0004FF002080EE04FF004080BE04FF04008E9
:1063C00008E04FF0080805E04FF0100802E04FF039
:1063D000200800BF00BF00BF33492068884201D1B8
:1063E000012000E0002000285DD00025B8F1100F4A
:1063F00033D009DCB8F1020F10D0B8F1040F11D07E
:10640000B8F1080F2ED117E0B8F1200F27D0B8F15E
:10641000400F0CD0B8F1800F24D124E0FCF7D6F85F
:10642000054623E005A8FCF7E7F8069D1EE002A854
:10643000FCF7F8F9039D19E01F4854380068C0F3D1
:10644000401040B11C4854380068C0F3C1012248D4
:1064500020FA01F500E0204D08E0204D06E04FF461
:10646000004503E000BF0120089000BF00BF002DE1
:106470000AD0606800EB4000A84203D860680003BF
:10648000A84202D201200890D4E2B8F1100F7CD0CB
:1064900026DCB8F1020F2DD0B8F1040F52D0B8F1BC
:1064A000080F73D19EE03FE1000C0058F369FFCF65
:1064B000FFF4FF1100100140544402580044004012
:1064C00000480040004C00400050004000140140D3
:1064D00000780040007C00400090D00300093D009F
:1064E000B8F1200F7DD0B8F1400F54D0B8F1800F33
:1064F000D7D109E1FCF76AF800270646FB49606A34
:1065000031F810C062463B4630463946F9F7E0FEA6
:106510004FF4807600220346A3FB060701FB0671B9
:1065200003FB021361684908064671185A41CDE918
:10653000001266683246002308460199F9F7C8FE42
:106540000546E4E005A8FCF757F8DDF818C0E74970
:10655000606A31F810B05A46002360461946F9F7D0
:10656000B7FE4FF4807C0022A0FB0C3B01FB0CB17A
:1065700000FB0210616849085E1840EB0201D4F884
:1065800004C062460023304601E079E0BBE0F9F741
:106590009FFE0546BBE002A8FCF744F9DDF80CC0FD
:1065A000D249606A31F810B05A4600236046194655
:1065B000F9F78EFE4FF4807C0022A0FB0C3B01FB20
:1065C0000CB100FB0210616849085E1840EB020143
:1065D000D4F804C0624600233046F9F779FE054638
:1065E00095E06EE0C2480068C0F3401038B3C04880
:1065F0000068C0F3C101BF4820FA01FCBB49606AD2
:1066000031F810B05A46002360461946F9F760FE8B
:106610004FF4807C0022A0FB0C3B01FB0CB100FB83
:106620000210616849085E1840EB0201D4F804C00A
:10663000624600233046F9F74BFE05461FE0AB49A2
:10664000606A31F810C062460023AA481946F9F77B
:106650003FFE4FF4807C0022A0FB0C3B01FB0CB101
:1066600000FB0210616849085E1840EB0201D4F893
:1066700004C0624600233046F9F72AFE054646E08C
:106680009A49606A31F810C0624600239A48194658
:10669000F9F71EFE4FF4807C0022A0FB0C3B01FBAF
:1066A0000CB100FB0210616849085E1840EB020162
:1066B000D4F804C0624600233046F9F709FE0546C7
:1066C00025E08A49606A31F810C0624600234FF421
:1066D00000401946F9F7FCFD4FF4807C0022A0FB36
:1066E0000C3B01FB0CB100FB0210616849085E180D
:1066F00040EB0201D4F804C0624600233046F9F7AB
:10670000E7FD054603E000BF0120089000BF00BF81
:10671000B5F5407F05D3B5F5801F02D22068C5606E
:1067200088E10120089085E1E069B0F5004F7CD157
:10673000B8F1100F7AD00CDCB8F1000F13D0B8F11B
:10674000010F21D0B8F1040F2FD0B8F1080F6ED18E
:1067500051E0B8F1200F6BD0B8F1400F38D0B8F14C
:10676000800F64D197E0FDF753F8604A616A32F810
:106770001110B0FBF1F04000616800EB5100B0FB7C
:10678000F1F01FFA80FA89E0FDF758F8574A616A7C
:1067900032F81110B0FBF1F04000616800EB5100DD
:1067A000B0FBF1F01FFA80FA78E005A8FBF724FFB0
:1067B00006994E4A606A32F81000B1FBF0F04000D2
:1067C000616800EB5100B0FBF1F01FFA80FA65E060
:1067D00002A8FCF727F80399444A606A32F81000CF
:1067E000B1FBF0F04000616800EB5100B0FBF1F04C
:1067F0001FFA80FA52E03E480068C0F34010C0B172
:106800003B480068C0F3C1013A48C840374A616A52
:1068100032F81110B0FBF1F04000616800EB51005C
:10682000B0FBF1F01FFA80FA12E044E011E031E031
:106830001FE02E49606A31F810002E49B1FBF0F0DC
:106840004000616800EB5100B0FBF1F01FFA80FAE4
:1068500024E02649606A31F810002749B1FBF0F0C6
:106860004000616800EB5100B0FBF1F01FFA80FAC4
:1068700014E01E49606A31F810004FF40041B1FB8A
:10688000F0F04000616800EB5100B0FBF1F01FFA3E
:1068900080FA03E000BF0120089000BF00BF4FF660
:1068A000F0700AEA0009CAF3420049EA00092068C8
:1068B000C0F80C90BEE0B8F1100F7CD00CDCB8F141
:1068C000000F1BD0B8F1010F29D0B8F1040F37D059
:1068D000B8F1080F70D159E0B8F1200F6DD0B8F1C0
:1068E000400F40D0B8F1800F66D19FE0C0980008FB
:1068F000004402580090D00300093D00FCF788FFD7
:106900004E4A616A32F81110B0FBF1F0616800EB99
:106910005100B0FBF1F080B22168C86089E0FCF75B
:106920008DFF464A616A32F81110B0FBF1F06168E0
:1069300000EB5100B0FBF1F080B22168C86078E054
:1069400005A8FBF759FE06993C4A606A32F8100028
:10695000B1FBF0F0616800EB5100B0FBF1F080B2E8
:106960002168C86065E002A8FBF75CFF0399334A21
:10697000606A32F81000B1FBF0F0616800EB510082
:10698000B0FBF1F080B22168C86052E02C4800688A
:10699000C0F34010C0B12A480068C0F3C1012948C3
:1069A000C840264A616A32F81110B0FBF1F0616804
:1069B00000EB510002E017E037E025E0B0FBF1F01A
:1069C00080B22168C8600EE01C49606A31F810008E
:1069D0001C49B1FBF0F0616800EB5100B0FBF1F035
:1069E00080B22168C86024E01449606A31F8100060
:1069F0001549B1FBF0F0616800EB5100B0FBF1F01C
:106A000080B22168C86014E00C49606A31F8100057
:106A10004FF40041B1FBF0F0616800EB5100B0FBB6
:106A2000F1F080B22168C86003E000BF0120089047
:106A300000BF00BF089809B0BDE8F08FC0980008FB
:106A4000004402580090D00300093D00014691F82F
:106A50007900212839D1B1F86200C8B90868006806
:106A600000F0005030B10868806820F400000B6826
:106A7000986005E00868006820F080000B681860E6
:106A80000868006840F040000B68186000207047FC
:106A90008868B0F5805F0BD1086948B9CA6D108865
:106AA000C0F308000B681885C86D801CC86505E038
:106AB000CB6D581CC86518780B681885B1F8620052
:106AC000401EA1F862000020E1E70220DFE72DE987
:106AD000F04104460D4617469846069E21E0701C7C
:106AE000F8B12EB1FAF7F0FCA0EB0800B04218D9CB
:106AF0002068006820F4D0702168086020688068F1
:106B000020F0010021688860202084F8790084F852
:106B10007A0000BF002084F8780000BF0320BDE8A1
:106B2000F0812068C0692840A84201D1012000E01E
:106B30000020B842D3D00020F1E7000070B5002457
:106B40000F4D1048FDF7ACFE00BF03E0641CAC42E3
:106B500000D904E00B48FDF799FE2028F6D100BFCC
:106B6000002403E0641CAC4200D906E0012206497F
:106B70000448FDF7FBFF0028F4D100BF70BD000002
:106B8000FFFF0100D40400241200002402460B463B
:106B9000D2F81812D2F8180218B10020C1F8140265
:106BA00070470220FCE770B504460E46D4F8185230
:106BB0003146204600F014FCC5F80C02D4F8180247
:106BC00048B1D5F80402D4F81C12CA6805F503715F
:106BD0009047002070BD0220FCE770B504460E46C9
:106BE00000258121204600F031FB0121204600F0E4
:106BF0002DFB8221204600F029FBD4F8180258B161
:106C0000D4F81C12486880470020D4F8181202F00B
:106C1000DBFD0020C4F81802284670BD70B505469B
:106C2000D5F81842D5F81C0278B194F80002FF2874
:106C30000BD094F8012294F80002D5F81C128B684E
:106C400021469847FF2084F80002002070BD000014
:106C500001460A20088001487047000020000024F7
:106C6000014643200880014870470000A800002426
:106C7000014643200880014870470000640000245A
:106C8000014643200880014870470000EC000024C2
:106C90002DE9F04104460F460026207C70B94FF4E0
:106CA000007302228121204600F0F8FB4FF40073AC
:106CB00002220121204600F0F1FB0BE040230222DA
:106CC0008121204600F0EAFB4023022201212046D8
:106CD00000F0E4FB082303228221204600F0DEFBC3
:106CE0004FF40771002002F081FDC4F81802D4F8B7
:106CF000180208B901261CE0D4F81852D4F81C1266
:106D0000086880470020C5F81402C5F81802207CE6
:106D100040B94FF4007301212046D5F8042200F059
:106D2000CDFB06E0402301212046D5F8042200F0E7
:106D3000C5FB3046BDE8F08170B50446D4F8185262
:106D4000D4F8180298B1207C40B94FF400730121A7
:106D50002046D5F8042200F0B1FB06E040230121D3
:106D60002046D5F8042200F0A9FB002070BD0220C7
:106D7000FCE70246022011B1C2F81C120020704745
:106D80000246D2F81832C3F804120020704710B53A
:106D90000346D3F81842C4F80812C4F810220020A1
:106DA00010BD000070B505460C46D5F81862207875
:106DB00000F0600040B3202835D1E088E0B12078B1
:106DC00000F0800060B1E2886078D5F81C128B6812
:106DD00031469847E2883146284600F0B9F812E07B
:106DE000607886F80002A07986F80102E2883146D0
:106DF000284600F08CF806E06078D5F81C120022D6
:106E00008B68214698470FE060780A2802D00B284B
:106E100007D105E001220649284600F099F800E074
:106E200000BF00BF00BF00BF00BF002070BD00005A
:106E30002F01002470B50546D5F81842D5F8180280
:106E400090B1D4F8140268B90120C4F81402B4F85F
:106E5000100283B281212846D4F8082200F0DFFB1B
:106E6000002070BD0120FCE70220FAE770B504465F
:106E70000D46D4F814022946426820469047002067
:106E800070BD70B504460D4694F8FC01022802D08E
:106E9000032811D100E000BF688801280BD1002031
:106EA000C4F80402D4F814022946826820469047A8
:106EB000204600F05EF804E02946204600F01BF86A
:106EC00000BF00BF70BD70B506460C4615462B4688
:106ED00022460021304600F0F1FA002070BD70B566
:106EE00006460C4615462B4622460021304600F049
:106EF00096FB002070BD70B504460D4680212046EB
:106F000000F071FB0021204600F06DFB70BD70B5F4
:106F100004460E4615460320C4F8F4014FF484706D
:106F20000551001D05512B4632460021204600F038
:106F3000C5FA002070BD10B504460520C4F8F40160
:106F400000231A461946204600F0B8FA002010BD6A
:106F500070B504460E4615460220C4F8F401A5613A
:106F6000E5612B4632460021204600F058FB002008
:106F700070BD10B504460420C4F8F40100231A467D
:106F80001946204600F04BFB002010BD70B50446AA
:106F90000D46E888012804D029462046FFF7ABFFBC
:106FA0001BE094F8FC01022802D003280FD108E06E
:106FB0000020A060012204F108012046FFF7C8FF6D
:106FC0000AE00122211D2046FFF7C2FF04E0294606
:106FD0002046FFF790FF00BF00BF70BDF8B5044624
:106FE0000E467088001208287FD2DFE800F07E0489
:106FF0000C207E7E5F6D207CD4F810120A686946F2
:107000009047054676E0207C40B9D4F81402816AA6
:107010006846884705460221697007E0D4F81402E3
:10702000C16A6846884705460221697062E0B07807
:10703000062834D2DFE800F0030B131B232B207C3F
:10704000D4F810124A686946904705462CE0207C27
:10705000D4F810128A6869469047054624E0207CDF
:10706000D4F81012CA686946904705461CE0207C97
:10707000D4F810120A6969469047054614E0207C4E
:10708000D4F810124A696946904705460CE0207C06
:10709000D4F810128A6969469047054604E03146E3
:1070A0002046FFF728FFF8BD00BF23E0207C30B961
:1070B000D4F81402416B6846884705461AE0314609
:1070C0002046FFF718FFEEE7207C48B9D4F81402F9
:1070D000016B684688470546072169700AE004E0AD
:1070E00031462046FFF707FFDDE731462046FFF730
:1070F00002FFD8E700BFBDF8000088B1F08878B182
:10710000F088BDF80010884202DDBDF8000000E004
:10711000F0880090BDF8002029462046FFF718FFB0
:1071200000BFC0E70146002002E0421CD0B2491C6B
:107130000A78002AF9D1704770B504460D4694F8D4
:10714000FC01022802D0032811D100E000BF012079
:10715000E060D4F8040218B1E06840F00200E0609A
:10716000022204F10C012046FFF7F2FE04E029465A
:107170002046FFF7C0FE00BF00BF70BD2DE9F04103
:1071800004460D4617460026FCB12046FFF7CAFF0D
:10719000022101EB400038803A783046711CCEB2B3
:1071A0002A5403223046711CCEB22A540AE014F845
:1071B000012B3046711CCEB22A5400223046711C7D
:1071C000CEB22A5420780028F1D1BDE8F081000029
:1071D00070B504460D46164654B90EA001F048FBA2
:1071E0000EA001F045FB13A001F042FB022070BD90
:1071F000D4F8140210B10020C4F814020DB1C4F880
:107200001052012084F8FC012670204600F0F2F8AC
:107210000020ECE74552524F523A2000496E766109
:107220006C6964204465766963652068616E646C8E
:10723000650000000D0A000070B504460D462946A1
:10724000D4F82002FAF720FB002070BD70B5044688
:107250000D462946D4F82002FAF7E0FA002070BD66
:107260002DE9F04104460E461746002E54D104F194
:107270001405D4F8F401022843D1D5E9020188426B
:1072800010D9D5E90201401AA860288982B239468E
:107290002046FFF724FE00231A461946204600F038
:1072A0000DF92EE0E9686868B0FBF1F201FB12000D
:1072B000B8B9E9686868884213D36868D4F8F811E7
:1072C00088420ED2002211462046FFF708FE002019
:1072D000C4F8F80100231A461946204600F0EEF8DB
:1072E0000FE0D4F81402C06840B194F8FC01032800
:1072F00004D1D4F81402C168204688472046FFF71D
:107300001AFE94F80002012814D1204600F0D2F9A8
:10731000002084F800020DE0D4F81402406948B15E
:1073200094F8FC01032805D1D4F8140231464269CF
:10733000204690470020BDE8F0812DE9F041054648
:107340000E4617465EBB05F58274D5F8F401032896
:1073500033D1D4E90201884210D9D4E90201401A9C
:10736000A060D4E90201884201D2A06800E0E06890
:1073700082B239462846FFF7A6FD1EE0D5F8140272
:10738000006940B195F8FC01032804D1D5F8140236
:107390000169284688472846FFF7EBFD0DE0D5F840
:1073A0001402806948B195F8FC01032805D1D5F88D
:1073B000140231468269284690470020BDE8F081DA
:1073C00001460020704710B50446012084F8FC01F6
:1073D0002179D4F81402426820469047002010BD5D
:1073E00070B504460D462946D4F82002FAF781FA12
:1073F00070BD000010B50446154816490860082005
:10740000486000211348016340214161002101626D
:10741000022181610021C1610221C1600021C1629C
:107420008162C0F8FC43C4F82002FAF7F9FE80211B
:107430000848FAF77AF9402200210648FAF77AF963
:10744000802201210348FAF775F9002010BD0000E1
:1074500000000840DC05002410B50246D2F82032B6
:1074600001F08000802809D101F07F00C0EBC0044A
:1074700003F1380000EB8400807810BD01F07F003C
:10748000C0EBC00403F5FC7000EB84008078F4E7E7
:107490000246002070470246002070472DE9F04167
:1074A00004460F4615461E462B4632463946D4F84A
:1074B0002002FAF72AFA0020BDE8F0812DE9F04118
:1074C00004460D4616461F463B4632462946D4F82A
:1074D0002002FAF761FA0020BDE8F08110B50446F9
:1074E0004023002211462046FFF7D8FF40214FF4E9
:1074F000887001514023002280212046FFF7CEFFF3
:1075000040212162012084F8FC01D4F8180228B13E
:107510002179D4F81402426820469047002010BD1B
:10752000014691F8FD0181F8FC010020704710B57B
:10753000044694F8FC01032808D1D4F81402C06969
:1075400020B1D4F81402C16920468847002010BD3C
:10755000024611740020704770B504460D460120A4
:10756000044908702946D4F82002FAF7BEFF00202B
:1075700070BD00003101002470B504460D46294657
:1075800004F5027000F05BF80120C4F8F40140F249
:107590000E20005BC4F8F80194F8080200F01F0008
:1075A00020B1012808D0022812D10BE004F50271A5
:1075B000204600F046F913E004F50271204600F081
:1075C00024FA0DE004F50271204600F073F907E09B
:1075D00094F8080200F08001204600F004F800BF93
:1075E00000BF002070BD70B504460D462946D4F892
:1075F0002002FAF7FEF9002070BD10B50446D4F859
:107600002002FAF794FF002010BD014691F8FC011A
:1076100081F8FD01042081F8FC01002070472DE96C
:10762000F04104460D4616461F463B463246294663
:10763000D4F82002FAF71BFA0020BDE8F0810A789E
:1076400002704A7842708B78CA7803EB022242803B
:107650000B794A7903EB022282808B79CA7903EB9A
:107660000222C2807047000070B505460C46002615
:1076700014B1C5F8144209E005A001F0F9F806A01C
:1076800001F0F6F80AA001F0F3F80226304670BDCA
:107690004552524F523A2000496E76616C6964201F
:1076A000436C6173732068616E646C650000000058
:1076B0000D0A000001460020704770B504460D46D3
:1076C000A888F8B9E888E8B9A87800F07F0694F8A7
:1076D000FC01032804D129462046FFF70CFC15E0E5
:1076E00084F8FE6131462046FFF736FF2046FFF75B
:1076F00040FC1EB1022084F8FC0107E0012084F860
:10770000FC0103E029462046FFF7F5FB70BD70B58C
:1077100004460D460226D4F8140238B1D4F81402F7
:10772000294602682046904700B90026304670BDC1
:1077300070B504460D46A8783449087008460078AC
:10774000012804DD29462046FFF7D5FB5BE094F8CD
:10775000FC01022802D003284FD11CE02B480078FE
:10776000A8B12A4800786060032084F8FC0127480B
:1077700001782046FFF7CBFF022804D12946204696
:10778000FFF7B9FB70BD2046FFF7F3FB02E0204690
:10779000FFF7EFFB36E01D48007870B9022084F84F
:1077A000FC011A4800786060184801782046FFF70D
:1077B0005DFB2046FFF7DDFB1EE014490978606899
:1077C000884216D021792046FFF750FB0F480078F9
:1077D00060600E4801782046FFF799FF022804D127
:1077E00029462046FFF787FBCCE72046FFF7C1FB81
:1077F00002E02046FFF7BDFB04E029462046FFF7E4
:107800007AFB00BF00BF00BFBCE7000030010024CE
:1078100070B504460D46688801280AD1C4F80402F0
:10782000D4F8140229468268204690472046FFF784
:10783000A0FB70BD10B504462046FFF7DEFE002019
:1078400010BD70B505460C46002660780A2829D27E
:10785000DFE800F01923281E280A0528140F214606
:107860002846FFF7BBFB22E021462846FFF725FF0D
:107870001DE021462846FFF75BFF18E02146284619
:10788000FFF784FB13E021462846FFF755FC0EE086
:1078900021462846FFF7BCFF09E021462846FFF7AE
:1078A000F0FA04E021462846FFF725FB00BF00BFA1
:1078B000304670BD2DE9F04105460E464FF00008F8
:1078C0003479307800F06000202808D1D5F814020F
:1078D00031468268284690470020BDE8F0817078E4
:1078E000002855D001282AD003287AD195F8FC0128
:1078F000022802D003281BD107E02CB1802C03D032
:1079000021462846FFF76FFE17E0708830B92CB18A
:10791000802C03D021462846FFF765FED5F81402D7
:1079200031468268284690472846FFF722FB04E04C
:1079300031462846FFF7DFFA00BF00BF62E095F846
:10794000FC01022802D003281BD107E02CB1802CB7
:1079500003D021462846FFF746FE17E0708878B925
:1079600004F07F0048B121462846FFF765FCD5F8B2
:10797000140231468268284690472846FFF7F9FAF4
:1079800004E031462846FFF7B6FA00BF00BF39E0F1
:1079900095F8FC01022802D003282BD107E004F05F
:1079A0007F0018B121462846FFF71DFE27E004F0AE
:1079B0008000802806D104F07F0105F1140000EB5F
:1079C000011005E004F07F0105F5827000EB011065
:1079D000074621462846FFF73FFD18B101203860D1
:1079E00002E00EE000203860022239462846FFF708
:1079F000AFFA04E031462846FFF77DFA00BF00BF2A
:107A000000E000BF00BF404667E770B504460D4682
:107A1000002694F8FC01032814D1287901280CDCF5
:107A2000D4F814022946826820469047E88840B975
:107A30003EB92046FFF79DFA03E029462046FFF7AE
:107A40005AFA04E029462046FFF755FA00BF00BF66
:107A5000002070BD70B505460C462DB9224606497A
:107A600006A0FFF78BFB04E02246034903A0FFF7C3
:107A700085FB014870BD0000DC09002456435020FE
:107A8000436F6E6669670000024612200880014855
:107A9000704700005001002470B505460C462DB912
:107AA0002246064906A0FFF769FB04E02246034987
:107AB00003A0FFF763FB014870BD0000DC09002450
:107AC00056435020496E746572666163650000001C
:107AD0000246042008800148704700006401002429
:107AE00070B505460C462246024903A0FFF746FB47
:107AF000004870BDDC09002453544D6963726F6502
:107B00006C656374726F6E696373000070B50546CF
:107B10000C462DB92246064906A0FFF72FFB04E0CC
:107B2000224603490CA0FFF729FB014870BD000065
:107B3000DC09002453544D33322056697274756148
:107B40006C20436F6D506F727420696E2048532013
:107B50004D6F64650000000053544D333220566968
:107B6000727475616C20436F6D506F727420696E12
:107B7000204653204D6F64650000000070B5054637
:107B80000C461A202080F9F7C1FA014870BD0000A8
:107B90006801002410B50246487801282BD140F630
:107BA0001C0080580C780123A3409BB2184340F678
:107BB0001C039850087802F5106303EB401000682E
:107BC00000F40040F0BB0889C0F30A00CB7840EA1B
:107BD00083400B7840EA835040F0805040F40040EE
:107BE00002F5106404EB43131B6818430B7804EB95
:107BF000431318602CE040F61C0080580C780123D9
:107C0000A340144C04EA0343184340F61C03985065
:107C1000087802F5306303EB4010006800F4004080
:107C200080B90889C0F30A00CB7840EA834040F06D
:107C3000805040F400400B7802F5306404EB4313AD
:107C40001B6800E004E018430B7804EB4313186052
:107C5000002010BD0000FFFF01464FF410604058A7
:107C6000C20AD2024FF41060425040F60800405859
:107C700000F00600042807D14FF41060405840F08F
:107C800003024FF41060425040F60400405840F4A4
:107C9000807240F604004250002070470FB410B5C7
:107CA00004460898012816D1A06B20F48030A06308
:107CB000E06815490840E060E06820F44010E060AA
:107CC0000F98012803D1E06840F48010E06020465E
:107CD00000F01CF809E0E06840F04000E060204659
:107CE00000F014F84FF48030A0630698012807D103
:107CF000A06840F00C00A060A06840F02000A060E8
:107D0000002010BC5DF814FBBFFFBDFF0146002240
:107D100000BF501C02460F4B984201D90320704708
:107D2000086900F000400028F3D00022086940F004
:107D30000100086100BF501C0246064B984201D961
:107D40000320ECE7086900F001000028F3D100BF30
:107D5000E5E70000400D030010B502464878012811
:107D600022D140F63C0080580C780123A3409BB2FE
:107D7000984340F63C03985040F61C0080580C781D
:107D80000123A3409BB2984340F61C039850087807
:107D900002F5106303EB4010006820F400440878FB
:107DA00003EB4010046026E040F63C0080580C785D
:107DB0000123A340114C04EA0343984340F63C03DB
:107DC000985040F61C0083580C780120A0400B4CC2
:107DD00004EA004023EA000040F61C0398500878AB
:107DE00002F5306303EB4010006820F4004408788B
:107DF00003EB40100460002010BD00000000FFFFF6
:107E000010B5044640F60400005920F0020140F687
:107E1000040001510320F9F709FA002010BD10B544
:107E2000044640F60400005940F0020140F6040008
:107E300001510320F9F7FAF9002010BD0FB430B555
:107E400004460025A06B40F40010A0630E9858B9BA
:107E5000A06B20F40010A063206840F04000206078
:107E6000206840F0800020600020C4F8000ED4F8A4
:107E70000008C4F80008099801280BD1069820B919
:107E80000021204600F078FC08E00121204600F0A7
:107E900073FC03E00321204600F06EFC1021204615
:107EA00000F0B4FB204600F09BFB00214FF4016082
:107EB0000151001D0151491E001D01510021001DED
:107EC0000151002524E004F5106000EB4510006826
:107ED00000F00040B0F1004F07D14FF0904104F5A1
:107EE000106000EB4510016005E0002104F5106012
:107EF00000EB45100160002104F5106000EB451017
:107F00000161FF2104F5106000EB451081606D1CDC
:107F10000498A842D7D8002524E004F5306000EB8F
:107F20004510006800F00040B0F1004F07D14FF05D
:107F3000904104F5306000EB4510016005E0002140
:107F400004F5306000EB45100160002104F530605D
:107F500000EB45100161FF2104F5306000EB451096
:107F600081606D1C0498A842D7D84FF40160005975
:107F700020F480714FF401600151079801280BD162
:107F800015494FF4036001510059144908434FF457
:107F900003610851084605590020A0616FF0804038
:107FA0006061079818B9A06940F01000A061A0694D
:107FB0000B490843A0610A9818B1A06940F0080075
:107FC000A0610E98012803D1A06906490843A06169
:107FD000002030BC5DF814FB00040002030001081F
:107FE00000383C80040000400146886820F0010011
:107FF000886000207047000030B5034648780128AB
:108000007DD1486918BB087803F5106404EB401073
:108010000069644C20400C7803F5106505EB4414AE
:10802000206108782C4604EB4010006940F40025DC
:10803000087804EB40100561087804EB40100069F3
:10804000C50CED04087804EB4010056137E00878B2
:1080500003F5106404EB40100069C50CED040878CA
:1080600004EB40100561087804EB401004694D48AA
:108070000440087803F5106505EB401004618C6836
:108080004869A04201D988684861087803F51064FE
:1080900004EB4010006940F40025087804EB401020
:1080A0000561087804EB401004694869C0F31200C8
:1080B0000443087803F5106505EB40100461012ABC
:1080C00007D1087803F5106404EB40100D69456191
:1080D0000BE0486948B140F63400C0580D780124DF
:1080E000AC40204340F63404E050087803F51064B7
:1080F00004EB4010006840F00445087800E003E01D
:1081000004EB401005604AE0087803F5306404EBA6
:1081100040100069C50CED04087804EB40100561BF
:10812000087804EB401000691E4C20400C7803F5E1
:10813000306505EB44142061486908B188684861DE
:10814000087803F5306404EB4010006940F4002522
:10815000087804EB40100561087804EB40100069D2
:108160008C68C4F3120420430C7803F5306505EBEA
:1081700044142061012A06D1087803F5306404EB29
:108180004010CD684561087803F5306404EB401079
:10819000006840F00445087804EB401005600020BA
:1081A00030BD0000FFFF07E010B503460024C3F810
:1081B000104BD3F8100B40F40024C3F8104BD3F845
:1081C000100B40F01804C3F8104BD3F8100B40F01C
:1081D000C044C3F8104B012906D1C3F8142B4FF04B
:1081E00080244FF43060C450002010BD10B502460A
:1081F000487801281ED1087802F5106303EB40107F
:10820000006820F40014087803EB40100460C8787C
:10821000032802D0C87802282AD1087802F5106312
:1082200003EB4010006840F08054087803EB4010E6
:1082300004601DE0087802F5306303EB401000682D
:1082400020F40014087803EB40100460C878032879
:1082500002D0C87802280BD1087802F5306303EB0E
:108260004010006840F08054087803EB4010046030
:10827000002010BD10B50246487801281FD10878AB
:1082800002F5106303EB4010006800F0004048B9AD
:10829000087803EB4010006820F08044087803EB76
:1082A00040100460087802F5106303EB401000688A
:1082B00040F40014087803EB401004601EE00878D6
:1082C00002F5306303EB4010006800F0004048B94D
:1082D000087803EB4010006820F08044087803EB36
:1082E00040100460087802F5306303EB401000682A
:1082F00040F40014087803EB40100460002010BD27
:10830000F8B505460C4616460027607801287DD151
:10831000606918BB207805F5106101EB4010006919
:10832000AA490840217805F5106202EB4111086165
:108330002078114601EB4010006940F400222078BB
:1083400001EB40100261207801EB40100069C20C83
:10835000D204207801EB401002614FE0207805F54F
:10836000106101EB40100069C20CD204207801EBCF
:1083700040100261207801EB4010006993490840E9
:10838000217805F5106202EB41110861A16860696E
:108390000844401EB0FBF1F08C49C94301EAC040DB
:1083A000217802EB411109690843217802EB411160
:1083B00008612078114601EB401001696069C0F343
:1083C00012000143207802EB40100161E07801289F
:1083D00014D12078114601EB4010006920F0C04212
:1083E000207801EB40100261207801EB4010006919
:1083F00040F00052207801EB40100261012E09D1BB
:10840000207805F5106101EB401000E04BE0226997
:1084100042610EE0E07801280BD0606948B140F677
:1084200034004059227801219140084340F634013C
:108430004851E07801281ED140F60800405900F468
:10844000807060B9207805F5106101EB401000687C
:1084500040F00052207801EB401002600BE02078E1
:1084600005F5106101EB4010006840F08052207863
:1084700001EB40100260207805F5106101EB40101F
:10848000006840F00442207801EB40100260E07880
:10849000012807D10096A08A83B222782846E16895
:1084A00000F072F98FE0207805F5306101EB4010A3
:1084B0000069C20CD204207801EB401002612078E0
:1084C00001EB4010016941480140207805F5306218
:1084D00002EB401001616069C0B92078114601EBE0
:1084E00040100069A168C1F312010843217802EB32
:1084F000411108612078114601EB4010006940F4F9
:108500000022207801EB4010026125E0A16860693B
:108510000844401EB0FBF1F087B2207805F53061C9
:1085200001EB401000692949C94301EAC7410843EA
:10853000217805F5306202EB41110861207811467F
:1085400001EB40100169A0687843C0F312000843B2
:10855000217802EB41110861012E06D1207805F542
:10856000306101EB4010E2684261E07801281ED1E1
:1085700040F60800405900F4807060B9207805F595
:10858000306101EB4010006840F00052207801EBB0
:10859000401002600BE0207805F5306101EB4010DF
:1085A000006840F08052207801EB40100260207893
:1085B00005F5306101EB4010006840F0044220787E
:1085C00001EB401002600020F8BD0000FFFF07E053
:1085D0000146886840F00100886000207047000074
:1085E000014600221020086100BF501C0246064BC5
:1085F000984201D903207047086900F01000102844
:10860000F3D00020F7E70000400D030010B502464C
:108610000023202040EA8110106100BF581C03464F
:10862000054CA04201D9032010BD106900F02000C4
:108630002028F3D00020F7E7400D0300014600207A
:1086400040F60802525802F0060202B917E040F65E
:108650000802525802F00602022A06D040F608022A
:10866000525802F00602062A01D1032007E040F624
:108670000802525802F00602042A00D10220704774
:108680000146486900F001007047014640F61800B5
:108690004258001D4058024090B27047014640F6D3
:1086A00018004258001D40580240100C704730B569
:1086B00002464FF40165AB5840F63405AC5824FA35
:1086C00001F505F0010543EAC51302F5106505EB58
:1086D0004115AD6805EA030030BD024602F530637E
:1086E00003EB4113986840F614039B5818407047F9
:1086F0000146002048698A691040704770B50346FA
:108700000024D01CC61700EB9676B51000BF05E01C
:108710004FF48050C0580860091D641CAC42F7D368
:10872000084670BD70B504460D46E06820F0C040B4
:10873000E060012D04D1E06840F00050E06004E00A
:108740001DB9E06840F08040E0603220F8F76EFD2F
:10875000002070BD0246D2F8000820F4FE60C2F886
:108760000008D2F800084FF4FE6303EA011318432F
:10877000C2F80008002070470246D2F800080843FB
:10878000C2F8000800207047F0B50446059E002797
:108790000025A6B9D81C4FEAE07C00EB9C7C4FEA90
:1087A000AC0700BF09E0D1F800C004F5805000EB31
:1087B0000230C0F800C0091D6D1CBD42F3D300207B
:1087C000F0BD00BFFEE7000030B503460C460022B6
:1087D00033E0995C1B48008800F4004058BB1948FE
:1087E000008800F4804060B10A2903D00020154DB4
:1087F000288020E01348008840F40040114D288074
:1088000019E00D2906D10F48008840F480400D4D35
:10881000288010E00B480088C0F30D000A4D295451
:1088200008480088401C074D288028460088C72833
:1088300001DD00202880501CC2B2A242C9D3002012
:1088400030BD00008C010024A40B002470B5044648
:108850000D46AAB221460548FEF799FA0348FEF7ED
:10886000E9FA012000F064FD70BD0000E801002479
:108870000FB4054B10B503A9044A029800F008F99B
:1088800010BC5DF814FB0000919300080C0000245C
:1088900037B514460846064B6A46214600F0A2F951
:1088A00004466946002000F034FD20463EBD00002D
:1088B0001393000802480068C0F3022070470000CC
:1088C0000CED00E010B5002804DB0A07130E054A82
:1088D000135406E00A07140E034A00F00F031B1F8F
:1088E000D45410BD00E400E018ED00E002E008C838
:1088F000121F08C1002AFAD170477047002001E01A
:1089000001C1121F002AFBD1704700002DE9FF5F53
:1089100082B00021DDE90430020DDDF840B00343F0
:1089200018D044F61050A2F2FF32424315141198A9
:1089300001281FD0A5EB0B00401C5FEA000A4FF096
:1089400000064E4FDFF83891B046504615D5CAF1B3
:10895000000413E0119801244AA3012801D16FEA11
:108960000B010298119AC0E90031C0E9024206B039
:10897000BDE8F09FCBF10000DFE704460021404A4C
:10898000491842EB0450CDE9001012E0E00707D08F
:1089900032463B4640464946F7F7C0FD8046894689
:1089A00032463B4610461946F7F7B8FD06460F46D5
:1089B0006410002CEAD1DDE90401DDE90023BAF1FD
:1089C000000F06DAF7F7AAFD42464B46F7F7A6FD79
:1089D00005E0F7F715FE42464B46F7F711FE044651
:1089E0000E460022284BF7F793FE03D84FF0FF30D6
:1089F000014607E00022254B20463146F7F7E7FC09
:108A0000F7F76DFE102409E0002C0ADB0A22002390
:108A1000F7F75EFC039B30321A55641E50EA0102E0
:108A2000F2D1641C039AC4F111031444119A012A6F
:108A300003D0012208430DD10AE0084304D00020EE
:108A40004FF0110B119072E7A3EB0B056D1E0DE0BB
:108A50005B4504DD4FF0000205F1010504E003DA97
:108A60004FF00002A5F10105002AECD002981199FF
:108A7000C0E90231C0E9004579E700000000144078
:108A80000000F03F300000000000F0430000E03F35
:108A90002DE9FF4F89B09B460446002506E02528B6
:108AA0000BD05A460B999047641C6D1C2078002807
:108AB000F5D10DB02846BDE8F08F0027B846012259
:108AC000474900E0074314F8013F203B02FA03F056
:108AD0000842F7D120782E2819D114F8010F47F059
:108AE00004072A280ED06FF02F022078A0F1300161
:108AF00009290CD808EB880102EB410100EB0108C1
:108B0000641CF2E70A98641C50F8048B0A902078E1
:108B10000028CED0642808D0692806D075281ED039
:108B20005A460B9990476D1C58E00A994FF00A0974
:108B300001C90A91002802DA40422D2102E03905DC
:108B400004D52B218DF82010012103E0F90704D072
:108B50002021F7E78A4608AE0DE00021FAE70A99DE
:108B60004FF00A0901C90A91F7E74946F7F7FAFBFE
:108B7000303106F8011D0028F7D1ADEB060000F1F9
:108B80002009780701D44FF00108C84502DDA8EBA1
:108B9000090000E000208046002706E008A85A46A9
:108BA000C05D0B9990476D1C7F1C5745F6DB04E0B8
:108BB00030205A460B9990476D1CB8F10001A8F17E
:108BC0000108F5DC05E016F8010B5A460B999047B1
:108BD0006D1CB9F10001A9F10109F4DC641C65E721
:108BE000092801002DE9FF4F95B09B4689460646AE
:108BF00000250FE2252877D100242746F84A0121D5
:108C0000059400E0044316F8013F203B01FA03F00D
:108C10001042F7D130782A2811D06FF02F03307826
:108C2000A0F13002092A16D8059A44F0020402EB9A
:108C3000820203EB42021044761C0590EFE759F8DC
:108C4000042B0592002A03DA504244F400540590A4
:108C500044F00204761C30782E2816D116F8010F45
:108C600044F004042A280DD06FF02F023078A0F1D0
:108C70003003092B09D807EB870302EB4303C7181E
:108C8000761CF3E759F8047B761C30786C280FD0FB
:108C900006DC4C2817D068280DD06A2814D104E0CF
:108CA000742810D07A280FD10DE044F400140AE0A3
:108CB00044F4801401E044F440147278824202D1FA
:108CC00004F58014761C761C307866280BD013DCF3
:108CD000582877D009DC002875D04528F6D04628DA
:108CE000F4D047281AD19DE118E0632835D06428D4
:108CF00079D0652812D195E1702873D008DC6728F7
:108D0000F1D069286FD06E280DD06F2806D1B5E05C
:108D100073282CD0752875D0782874D05A461799A6
:108D200090476D1C75E1C4F30250022809D0032856
:108D30000DD0D9F8001004280DD00D6009F10409F8
:108D400067E1D9F80010EA17C1E90052F6E7D9F84F
:108D500000100D80F2E70D70F0E719F8041B8DF894
:108D6000001000208DF80100EA46012003E059F8C8
:108D700004AB4FF0FF3061074FF0000102D40DE06B
:108D800008F101018846B9420FDA8045F8DB1AF88C
:108D900008100029F4D108E008F101018846814259
:108DA000FADB1AF808100029F6D105985B46A0EB0B
:108DB000080721463846179A00F094FA284400EB39
:108DC000080507E04DE029E10DE01AF8010B5A46CD
:108DD00017999047B8F10108F7D25B46214638460B
:108DE000179A13E142E00A220092C4F302524FF0B4
:108DF000000A022A08D059F804CB032A4FEAEC7182
:108E00000AD00DE029E02AE009F1070121F007026C
:108E1000F2E802C1914609E00FFA8CFC4FEAEC71CE
:108E2000042A03D14FFA8CFC4FEAEC71002907DACF
:108E30000A460021DCF1000C61EB02012D2202E068
:108E4000220504D52B228DF80420012203E0E2073D
:108E500001D02022F7E7904659E00A2102E01022D3
:108E60000DE010214FF0000A00910BE010224FF0AE
:108E7000000A44F004040827009203E008224FF09F
:108E8000000A0092C4F30252022A05D059F804CB1A
:108E90000021032A08D009E009F1070121F00702A7
:108EA000F2E802C1914605E01FFA8CFC042A01D1C8
:108EB0000CF0FF0C4FF00008220728D5702806D0D0
:108EC000009B83F0100353EA0A0305D00EE0402212
:108ED0008DF80420012208E05CEA010206D030226D
:108EE0008DF804208DF8050002229046009B83F047
:108EF000080353EA0A030AD15CEA010201D16207BE
:108F000005D530228DF804204FF001087F1E582827
:108F100004D034A003900EA802900DE036A0F9E72B
:108F200053466046009AF7F7D3F984460398825C6B
:108F30000298401E029002705CEA0100F0D1029893
:108F400006A9081A00F1200A600702D524F480342B
:108F500000E00127574502DDA7EB0A0000E00020F2
:108F600000EB0A01009005984144401A0590E00387
:108F700006D45B462146179A059800F0B3F90544DC
:108F8000002706E001A85A46C05D179990476D1C5E
:108F90007F1C4745F6DBE0030CD55B462146179A5C
:108FA000059800F09FF9054404E030205A461799CF
:108FB00090476D1C0099481E00900029F5DC08E0E0
:108FC000029802995A460078491C029117999047D5
:108FD0006D1CBAF10001AAF1010AF1DC65E10000A3
:108FE000092801003031323334353637383961627F
:108FF0006364656600000000303132333435363743
:1090000038394142434445460000000000F058F919
:109010000544761C307800287FF4ECAD19B0284662
:10902000BDE8F08F620700D4062709F1070222F09D
:10903000070CFCE80223E14603F000485FEA080C55
:1090400002D00FF2702C0DE05FEA045C02D50FF243
:10905000682C07E05FEAC47C02D00FF2602C01E0CC
:10906000AFF2700C4FF0FF3823F00043CDF850C042
:1090700065280CD006DC452809D046281DD0472895
:109080003DD13DE0662818D067287ED138E0002128
:10909000112F01DB112000E0781CCDE9000106A9A9
:1090A0000EA8FFF733FCDDE90F010E9A03910021B2
:1090B000009207F1010A04914DE04FF00040009743
:1090C000CDE9011006A90EA8FFF720FCDDE90F028B
:1090D00003920E9B11990022DDF80CA000930492DC
:1090E00011B9791C00EB010AB7EB0A0004D4C0F1F6
:1090F000FF3007F1010A0490AAEB0700019044E059
:10910000012F00DA01270021112F01DD112000E0DD
:109110003846CDE9000106A90EA8FFF7F7FBDDE907
:109120000F010E9A0391002104910092BA46210783
:109130000CD40399514500DA8A46BAF1010F05DDD6
:10914000009AAAF10101515C302908D0B84202DA34
:1091500010F1040F06DA0121CDE9011015E0AAF1A2
:109160000101E9E7002805DC049901440491AAEB18
:10917000000102E0411C514500DD8A460499401A75
:10918000401C01904FF000400290200704D4019849
:10919000504501DBCDF8048000208DF84F00029887
:1091A0000DF14F07B0F1004F25D02B200E90029803
:1091B0004FF0020800280CDA404202902D200E9059
:1091C00007E00A210298F7F7CDF83031029007F84E
:1091D000011DB8F10001A8F10108F2DC0298002895
:1091E000EFD1791E0E980870307800F0200040F022
:1091F000450007F8020D12A8C01B00F107081498DB
:10920000007800B1012000EB0A01019801EBE07148
:1092100005984144401A401E0590E00306D45B4681
:109220002146179A059800F05DF8054414980078D7
:1092300018B15A46179990476D1CE00324D55B4638
:109240002146179A059800F04DF805441CE0049853
:10925000002807DBDDE90301884203DD0098405C5C
:10926000179901E0179930205A469047049805F164
:109270000105401C04900198401E019004D12E204D
:109280005A46179990476D1CBAF10001AAF1010ADC
:10929000DDDC05E017F8010B5A46179990476D1C65
:1092A000B8F10001A8F10108F4DC5B462146179AE9
:1092B0000598ABE62D0000002B0000002000000008
:1092C0002DE9F041044600251E461746880404D4C3
:1092D00005E039462020B0476D1C641EF9D52846AC
:1092E000BDE8F0812DE9F041044600251E46904678
:1092F000C80301D5302700E02027880404D505E005
:1093000041463846B0476D1C641EF9D52846BDE875
:10931000F0810A68531C0B601070704710B504464A
:109320000420FBF783FA0148046010BD0800002404
:1093300030B50446002504E04FF47A7000F004F8DC
:109340006D1CA542F8D330BD70B5034600224FF026
:10935000E02675690D4E366803FB06F44FF0E026F3
:10936000B16910E04FF0E026B06988420BD0884226
:1093700002D20E1A324402E02E1A0E443244014642
:10938000A24200D300E0EDE700BF70BD080000245A
:1093900000BF054AD26902F04002002AF9D0C2B2E9
:1093A000014B1A8570470000001001400024002680
:1093B000F7F72EFBFCF72AF8F8F798F804230222B7
:1093C0000521A020FCF780FC4FF4C870FFF7A6FF32
:1093D0004FF4E13000F028FAFBF7F2FFFBF79CFCBA
:1093E000FBF7D0FDF7F7C0FC4FF6FF70FBF7D2FCA0
:1093F000002000F05FF9042000F05CF947A34FF46F
:10940000784210210846F7F79BFB4AA31F22202130
:109410001020F7F795FB4CA31F2230211020F7F7FF
:109420008FFB4EA31F2246211020F7F7A9FB002235
:109430004F495048FDF7CCFE4F494E48FEF714F90E
:109440004E494C48FDF795FC4A48FEF7F3F9F9F709
:1094500097F862E04A480078864221D0484806786A
:10946000012E0ED11F204749088047A31F22462105
:109470001020F7F785FB002202214848F8F71EF874
:109480000EE04FF478403F49088045A31F22462153
:109490001020F7F775FB012202214048F8F70EF87B
:1094A0004448008800F4004090B142480088C0F36E
:1094B0000D05294640A000F0D3F929464548FFF79D
:1094C000C5F945A000F0CCF900203A49088024E015
:1094D000601C84B241F2883094FBF0F100FB114033
:1094E00028B93FA000F0BCF948A000F0B9F9C820A5
:1094F00094FBF0F100FB114010B94CA000F0B0F962
:109500001E2094FBF0F100FB114018B90221234802
:10951000F7F7D0FF0A20FFF70BFF9BE720205354FB
:109520004D33324837205553422D55534152542024
:10953000000000002020C7B6C8EBCABDBFAAB7A272
:10954000CDF82020200000006D63756465762E74D0
:10955000616F62616F2E636F6D0000005553422092
:10956000436F6E6E656374696E672E2E2E00000069
:1095700034010024E80100242C0000249001002480
:1095800031010024E001002455534220436F6E6EE8
:1095900065637465642020202000000000000258EC
:1095A00055534220646973436F6E6E6563746564DE
:1095B000200000008C0100240D0AC4FAB7A2CBCD14
:1095C000B5C4CFFBCFA2B3A4B6C8CEAA3A25640DCA
:1095D0000A0D0A00A40B00240D0A0D0A0000000069
:1095E0000D0A202053544D333246342F46372F482E
:1095F00037BFAAB7A2B0E5555342D0E9C4E2B4AE32
:10960000BFDACAB5D1E90D0A00000000B4F3D4BD39
:10961000B4B4D0C22D6D63756465762E74616F62CB
:10962000616F2E636F6D200D0A0D0A00C7EBCAE44F
:10963000C8EBCAFDBEDD2CD2D4BBD8B3B5BCFCBDD3
:10964000E1CAF80D0A0000002DE9F04104460E467B
:109650001548005D38B914483838016820468847F5
:109660000120BDE8F081114850F82400B04219D91A
:109670000F4850F82400B6FBF0F10B48183850F8AA
:10968000240050F82120002508E00023064818385F
:1096900050F824004F1940F827306D1C9542F4DB38
:1096A0000020DEE70220DCE7D80100242099000832
:1096B0000899000810B50446074951F824108A009B
:1096C000064951F82400002100F0A4F801210348C4
:1096D0001830015510BD0000F0980008C0010024AA
:1096E0002DE9F04704460F460025A9462348005DB2
:1096F00020B9224838380168204688471FB94FF002
:10970000FF30BDE8F0871E4850F82400B7FBF0F6A4
:109710001B4850F82400B7FBF0F100FB117000B1BA
:10972000761C184850F82400451E22E013481838CB
:1097300050F8240050F8250010B909F1010901E0A2
:109740004FF00009B14513D14FF0000809E00B4874
:10975000183850F8240005EB080140F8216008F1A2
:109760000108B045F3D3064850F824006843C8E721
:109770006D1E002DDADA4FF0FF30C2E7D801002469
:1097800008990008F098000810B50146002300224F
:1097900007E00B4850F8210050F8220000B15B1C94
:1097A000521C084850F821009042F2D84FF47A70C9
:1097B0005843044C54F82140B0FBF4F080B210BD83
:1097C000C0010024F098000870B505460C4604B9A5
:1097D00070BD054850F82500261A31462846FFF787
:1097E00033FF00BFF4E70000A801002470B5044671
:1097F0000E4631462046FFF773FF0546681C08B940
:10980000002070BD024850F824002844F9E7000009
:10981000A801002430B5034601E003F8011B141E23
:10982000A2F10102F9D130BD10B5044609480A4938
:1098300008600846446000218160C1600161816167
:109840000C214161FBF70AF9012204490248FBF7A8
:109850008DF910BD00100140D40400241200002432
:109860000FB438B505A800900A48009A0499FFF78C
:109870000FF8002000900748F6F76DFD84B22146EE
:109880000448FEF7E3FF21460248FBF793FF38BC8C
:109890005DF814FBDC0A002401000200040006004D
:1098A00008000A000C0010002000400080000001A9
:1098B0000000000001020304010203040607080976
:1098C000010002000400060008000A000C0010005D
:1098D000200040008000000101000200040006009A
:1098E00008000A000C001000200040008000000169
:1098F0000010000001000000000F0000C003000085
:1099000080070000C003000040000000400000008D
:109910004000000040000000400000004000000047
:10992000000004004000000000C0030000F0000040
:1099300000E0010000F00000000000000000000056
:1099400000000000000000003F4000000000000098
:1099500000003000400030004000000009000BC053
:109960003D000BC03D00090018C024407FE02240AC
:1099700031800000180024C01B000D80324001809F
:1099800003801C4027401C800740004010006000FE
:1099900000000000000000000000000000001F8028
:1099A000204040200000402020401F800000000098
:1099B000090006001F8006000900000004000400E2
:1099C0003F80040004000000001000600000000060
:1099D0000000000004000400040004000400000073
:1099E000000000400000000000000000002001C056
:1099F00006003800400000001F802040204020402A
:109A00001F800000000010403FC000400000000028
:109A100018C02140224024401840000010802040FF
:109A2000244024401B80000002000D0011003FC0B4
:109A3000014000003C80244024402440238000005A
:109A40001F80244024403440038000003000200068
:109A500027C03800200000001B8024402440244000
:109A60001B8000001C0022C0224022401F800000FA
:109A7000000000000840000000000000000000009E
:109A80000460000000000000000004000A00110053
:109A90002080404009000900090009000900000079
:109AA00000004040208011000A000400180020003F
:109AB00023402400180000001F8020402740294038
:109AC0001F400000004007C039000F0001C00040E7
:109AD00020403FC0244024401B8000001F802040C5
:109AE000204020403080000020403FC020402040E7
:109AF0001F80000020403FC024402E4030C00000A6
:109B000020403FC024402E00300000000F00108095
:109B1000204022403380020020403FC00400040067
:109B20003FC02040204020403FC020402040000057
:109B30000060202020203FC02000200020403FC0A7
:109B400024400B0030C0204020403FC02040004057
:109B5000004000C03FC03C0003C03C003FC00000CC
:109B600020403FC00C4023003FC020001F80204009
:109B7000204020401F80000020403FC0244024009F
:109B8000180000001F802140214020E01FA000009D
:109B900020403FC02440260019C0004018C0244087
:109BA0002440224031800000300020403FC020404F
:109BB0003000000020003F80004000403F80200037
:109BC00020003E0001C0070038002000380007C018
:109BD0003C0007C038000000204039C0060039C0F2
:109BE000204000002000384007C03840200000001E
:109BF000304021C02640384020C000000000000056
:109C00007FE0402040200000000070000C00038036
:109C1000004000000000402040207FE000000000E5
:109C20000000200040002000000000000010001094
:109C300000100010001000100000000040000000A4
:109C400000000000000002800540054003C0004005
:109C500020003FC004400440038000000000038057
:109C600004400440064000000000038004402440FB
:109C70003FC0004000000380054005400340000055
:109C8000000004401FC0244024402000000002E0E7
:109C9000055005500650042020403FC004400400F9
:109CA00003C000400000044027C000400000000046
:109CB00000100010041027E00000000020403FC00A
:109CC0000140070004C00440204020403FC0004045
:109CD0000040000007C0040007C0040003C00000EB
:109CE000044007C00440040003C00040000003809B
:109CF0000440044003800000041007F004500440B6
:109D000003800000000003800440045007F00010AE
:109D1000044007C0024004000400000000000640A8
:109D20000540054004C00000000004001F800440FE
:109D300000400000040007800040044007C00040CD
:109D40000400070004C0018006000400060001C0F2
:109D5000070001C006000000044006C0010006C064
:109D6000044000000410071004E001800600040015
:109D70000000044005C00640044000000000000050
:109D800004007BE040200000000000000000FFF025
:109D900000000000000040207BE004000000000004
:109DA0004000800040002000200040000000000033
:109DB00000000000000000000000000000000000A3
:109DC00000001FCC000C0000000000000000080094
:109DD000300060000800300060000000022003FC3A
:109DE0001E20022003FC1E200220000000000E188E
:109DF00011043FFF10840C78000000000F00108455
:109E00000F3800C0077818840078000000780F84AD
:109E100010C411240E9800E40084000808006800B3
:109E200070000000000000000000000000000000C2
:109E3000000007E018182004400200000000400263
:109E40002004181807E00000000000000240024053
:109E500001800FF00180024002400000008000807D
:109E600000800FF800800080008000000001000DDD
:109E7000000E000000000000000000000000008054
:109E80000080008000800080008000800000000CC6
:109E9000000C0000000000000000000000000006B0
:109EA000001800600180060018002000000007F084
:109EB000080810041004080807F000000000080457
:109EC00008041FFC000400040000000000000E0C49
:109ED00010141024104411840E0C000000000C1803
:109EE00010041104110412880C700000000000E03E
:109EF0000320042408241FFC0024000000001F98F5
:109F0000108411041104108810700000000007F084
:109F100008881104110418880070000000001C005B
:109F2000100010FC13001C001000000000000E3890
:109F300011441084108411440E3800000000070002
:109F4000088C10441044088807F00000000000004E
:109F50000000030C030C00000000000000000000E3
:109F60000001010600000000000000000000008069
:109F70000140022004100808100400000220022002
:109F80000220022002200220022000000000100413
:109F900008080410022001400080000000000E00AC
:109FA0001200100C106C10800F00000003E00C1861
:109FB00013E4142417C4082807D000000004003C50
:109FC00003C41C40074000E4001C000410041FFCF4
:109FD0001104110411040E880070000003E00C1835
:109FE00010041004100410081C10000010041FFCC2
:109FF000100410041004080807F0000010041FFCEF
:10A000001104110417C410040818000010041FFCE8
:10A010001104110017C010000800000003E00C1824
:10A020001004100410441C780040000010041FFCB1
:10A0300010840080008010841FFC100400001004B5
:10A0400010041FFC100410040000000000030001B5
:10A05000100110011FFE10001000000010041FFC72
:10A06000110403801464181C1004000010041FFC69
:10A070001004000400040004000C000010041FFC85
:10A080001F0000FC1F001FFC1004000010041FFC38
:10A090000C04030000E010181FFC100007F0080873
:10A0A000100410041004080807F0000010041FFC3E
:10A0B00010841080108010800F00000007F0081836
:10A0C00010241024101C080A07F2000010041FFCC2
:10A0D0001104110011C011300E0C000400000E1C00
:10A0E00011041084108410441C3800001800100063
:10A0F00010041FFC100410001800000010001FF8CE
:10A1000010040004000410041FF8100010001E00CA
:10A1100011E0001C007013801C0010001FC0103CD8
:10A1200000E01F0000E0103C1FC000001004180CED
:10A13000163401C001C01634180C100410001C00A5
:10A14000130400FC13041C00100000000804101C81
:10A150001064108413041C04101800000000000098
:10A1600000007FFE4002400240020000000030007C
:10A170000C0003800060001C00030000000040028F
:10A18000400240027FFE00000000000000000000CE
:10A1900020004000400040002000000000010001BD
:10A1A0000001000100010001000100010000400069
:10A1B00040002000000000000000000000000098A7
:10A1C000012401440144014400FC000410001FFC70
:10A1D0000088010401040088007000000000007085
:10A1E00000880104010401040088000000000070E0
:10A1F00000880104010411081FFC0004000000F89D
:10A20000014401440144014400C80000000001046D
:10A2100001040FFC1104110411001800000000D605
:10A2200001290129012901C90106000010041FFCB0
:10A23000008401000100010400FC0004000001048E
:10A24000190419FC000400040000000000000003D1
:10A2500000010101190119FE0000000010041FFC9B
:10A260000024004001B4010C0104000000001004AF
:10A2700010041FFC0004000400000000010401FCA5
:10A280000104010001FC0104010000FC010401FCC7
:10A29000008401000100010400FC0004000000F83B
:10A2A000010401040104010400F80000010101FFA0
:10A2B00000850104010400880070000000000070A7
:10A2C000008801040104010501FF000101040104EB
:10A2D00001FC00840104010001800000000000CCAA
:10A2E0000124012401240124019800000000010040
:10A2F000010007F80104010400000000010001F85A
:10A30000000400040004010801FC000401000180B5
:10A310000170000C001001600180010001F0010CCF
:10A32000003001C00030010C01F001000000010408
:10A33000018C00740170018C010400000101018195
:10A340000171000E0018016001800100000001840D
:10A35000010C013401440184010C000000000000E4
:10A360000000000001003EFC40024002000000002E
:10A3700000000000FFFF000000000000000040029D
:10A3800040023EFC010000000000000000006000F0
:10A3900080008000400040002000200000000000FD
:10A3A00000000000000000000000000000000000AD
:10A3B000000000000000000000000000000000009D
:10A3C0000000000000000000000000000000000F7E
:10A3D00080380FFE380F80380000000000000000B9
:10A3E0000000000000000000000001000006000066
:10A3F0000C00003800003100000600000C0000389E
:10A4000000003000000000000000000061800067D4
:10A41000F807F98000618000618000618000618040
:10A420000067F807F980006180000000000000006C
:10A43000000001C0E003E0F00630080418081FFF28
:10A44000FE040E080787F00381E000000000000012
:10A4500001F000060C00040408060C7001F9C000AD
:10A460000E00003BE000EC18070808040C1800037D
:10A47000E00000000001E00007F003F818041C08E9
:10A4800004170807E1D003C0E00023B0003C080037
:10A490002008000010000000000000010000310052
:10A4A000003200001C00000000000000000000005E
:10A4B000000000000000000000000000000000009C
:10A4C0000000000000000000000000007F0001FF0D
:10A4D000C00780F00C0018100004200002000000EB
:10A4E0000000002000021000040C00180780F0019A
:10A4F000FFC0007F0000000000000000000000001E
:10A50000000000000000000042000066000066003D
:10A51000003C0000180003FFC0001800003C0000D1
:10A52000660000660000420000000000080000080D
:10A530000000080000080000080001FFC00008003B
:10A5400000080000080000080000080000000000EB
:10A55000000100003100003200001C00000000007B
:10A5600000000000000000000000000000000000EB
:10A5700000000000080000080000080000080000BB
:10A58000080000080000080000080000080000089B
:10A59000000000000000000000000000380000384B
:10A5A0000000380000000000000000000000000073
:10A5B0000000000000000000000000000006000095
:10A5C0001C000070000180000E0000380000C00078
:10A5D0000700001C00003000000000000000000028
:10A5E0007F8001FFE003807006001804000804006B
:10A5F0000806001803807001FFE0007F8000000063
:10A60000000000000000010008010008010008032C
:10A61000FFF807FFF800000800000800000800002D
:10A620000000000000000001C03802C0580400987B
:10A63000040118040218040418061C1803F8180171
:10A64000E0F800000000000000000001C0E003C0CE
:10A65000F004000804080804080806180803F418A1
:10A6600001E7F00001E00000000000000000000031
:10A670000300000D000011000061000081080301CB
:10A680000807FFF80FFFF8000108000108000000AC
:10A690000000000000E007FCD006080806100806CD
:10A6A0001008061008061838060FF00607C000004C
:10A6B00000000000000000003F8001FFE003843044
:10A6C00002081804100804100804100807181003E2
:10A6D0000FF00007C000000000000000000003C0F1
:10A6E000000700000600000600F80607F80618003C
:10A6F00006E0000700000600000000000000000166
:10A70000E1E003F7F0063410041808041808040CFC
:10A7100008040C0806161803F3F001C1E00000005D
:10A7200000000000F80003FC3003063804020804AF
:10A7300002080402080404100308F001FFC0007FAF
:10A740000000000000000000000000000000000009
:10A750000000000070380070380070380000000001
:10A7600000000000000000000000000000000000E9
:10A770000000000000000000301A00301C00000043
:10A7800000000000000000000000000000000000C9
:10A7900000000008000014000022000041000080BA
:10A7A00080010040020020040010080008000000A2
:10A7B0000000000021000021000021000021000015
:10A7C00021000021000021000021000021000021C3
:10A7D0000000000000000000000008000804001055
:10A7E00002002001004000808000410000220000A3
:10A7F000140000080000000000000003C00004C0B6
:10A8000000040000080038080F3808083808100055
:10A810000C300007E00003C0000000000000000052
:10A820003F8000FFE0038070020F1006708804C0B4
:10A8300088048308047F8802C09003012000FE4042
:10A840000000080000180001F8003E0801C20007DF
:10A85000020007E20000FE00001FC80001F800002F
:10A860003800000804000807FFF807FFF80408088C
:10A8700004080804080804080806180803F4180166
:10A88000E7F00001E0000000000000003F8001FF51
:10A89000E0038070020018040008040008040008A7
:10A8A0000400100600200780C00000000400080714
:10A8B000FFF807FFF804000804000804000804007B
:10A8C0001802001003807001FFE0007F800000008C
:10A8D00004000807FFF807FFF80408080408080444
:10A8E0000808040808043E080400080600180100CF
:10A8F0006000000004000807FFF807FFF8040808DC
:10A90000040800040800040800043E0006000006D5
:10A910000000018000000000000000003F8001FFF7
:10A92000E00380700600180400080402080402080E
:10A930000203F00783F00002000002000400080791
:10A94000FFF807FFF80408080008000008000008E6
:10A950000000080004080807FFF807FFF8040008D3
:10A9600000000000000004000804000804000807BC
:10A97000FFF807FFF80400080400080400080000BE
:10A9800000000000000000000006000007000001B9
:10A9900004000104000104000307FFFE07FFFC049C
:10A9A000000004000004000004000807FFF807FF8F
:10A9B000F8040C08001800003E0004C7800503C816
:10A9C0000600F80400380400180000080400080716
:10A9D000FFF807FFF8040008000008000008000066
:10A9E00008000008000008000018000060000000D7
:10A9F00004000807FFF807800807FC00007FC0007C
:10AA000003F80007C000780007800807FFF807FF79
:10AA1000F804000804000807FFF807000803C00056
:10AA200000E000003800001E000007000001C00424
:10AA300000F007FFF8040000000000007F8001FF25
:10AA4000E0038070060018040008040008060018DF
:10AA500003003001FFE0007F8000000004000807D1
:10AA6000FFF807FFF80404080404000404000404C9
:10AA700000040400060C0003F80001F000000000D0
:10AA8000000000007F8001FFE00380700600880462
:10AA900000880400C806003C03003E01FFE6007F7A
:10AAA0008400000004000807FFF807FFF804080806
:10AAB000040800040C00040F00040BC00610F0038F
:10AAC000F03801E00800000800000001E0F803F0A1
:10AAD00030063010041808041808040C08040C0888
:10AAE0000206180207F00781E0000000018000065E
:10AAF000000004000004000004000807FFF807FF3E
:10AB0000F8040008040000040000060000018000B2
:10AB100004000007FFE007FFF00400180000080031
:10AB2000000800000800000800000804001007FFEB
:10AB3000E004000004000006000007E00007FE003B
:10AB4000041FE00001F80000380001E0043E0007A7
:10AB5000C00006000004000004000007E00007FF3A
:10AB6000C0041FF80007C007F80007FF80043FF883
:10AB70000007C004F8000700000400000000000403
:10AB8000000806001807C07805F1C8003E00001F45
:10AB9000800463E80780F80600180400080000003D
:10ABA00004000006000007800007E008047C08009D
:10ABB0001FF80007F800180804E008070000060066
:10ABC000000400000000000100080600380400F83E
:10ABD0000403E8040F08047C0805F00807C0080710
:10ABE00000180400600000000000000000000000E9
:10ABF000000000000000003FFFFE200002200002D5
:10AC000020000220000220000200000000000000DE
:10AC1000000008000007000000C000003800000627
:10AC2000000001C000003000000E00000100000024
:10AC3000000000000000200002200002200002208E
:10AC400000022000023FFFFE0000000000000000A4
:10AC500000000000000000000000000000080000EC
:10AC6000100000300000200000300000100000083C
:10AC700000000000000000000000010000010000D2
:10AC800001000001000001000001000001000001BE
:10AC900000000100000100000100000100000000B0
:10ACA0000000000000200000200000100000100044
:10ACB0000000000000000000000000000000000094
:10ACC0000000000000F00019F8001B180022080026
:10ACD0002608002408002410003FF8001FF8000098
:10ACE0000800001800000004000007FFF80FFFF044
:10ACF0000018180010080020080020080030180074
:10AD00001FF0000FC00000000000000007C0001F7F
:10AD1000F0001830002008002008002008003C083F
:10AD2000001C100000600000000000000000000097
:10AD300007C0001FF000381800200800200800207D
:10AD40000804101007FFF80FFFF0000010000000CB
:10AD50000000000000000007C0001FF000123000DB
:10AD60002218002208002208003208001E10000EDF
:10AD70002000000000000000200000200800200843
:10AD800001FFF803FFF80620080420080420080744
:10AD9000200003000000000000000000000E000E74
:10ADA0006E001FF30031B10020B10020B1003191DD
:10ADB000001F13002E1E00200E00300000000004B3
:10ADC000000807FFF80FFFF800100800200000201F
:10ADD00000002008003FF8001FF8000008000000F5
:10ADE00000000000000000200800200800200806E5
:10ADF0003FF8063FF80000080000080000080000C7
:10AE0000000000000000000000000000030000033C
:10AE1000002001002001002003063FFE063FFC0049
:10AE2000000000000000000000000004000807FF10
:10AE3000F80FFFF8000188000300002FC00038F869
:10AE4000002038002008000008000000000000007A
:10AE5000000004000804000804000807FFF80FFFC2
:10AE6000F8000008000008000008000000000000D2
:10AE7000002008003FF8003FF80010080020000004
:10AE80003FF8003FF8001008002000003FF8003FA6
:10AE9000F8000008000000002008003FF8003FF81C
:10AEA000001008001000002000002008003FF800FB
:10AEB0001FF80000080000000000000007C0000F9D
:10AEC000F00018300030080020080020080030088A
:10AED000001830000FF00007C00000000000000064
:10AEE0002001003FFF003FFF00101100200900205B
:10AEF00008002008003038001FF0000FC0000000DC
:10AF00000000000007C0001FF000381800200800F3
:10AF10002008002009001011001FFF003FFF000063
:10AF200001000000002008002008002008003FF871
:10AF3000003FF8000808001008002008002000006A
:10AF40003000003000000000000000000000000C95
:10AF500078001E180033080023080021080021880B
:10AF60000021980030F00038600000000000000070
:10AF7000200000200000200000FFF003FFF8002068
:10AF80000800200800200800003000000000000039
:10AF9000000000002000003FF0007FF800001800D3
:10AFA0000008000008002010003FF8007FF00000BB
:10AFB00010000000000000002000003000003C00F5
:10AFC000003F800023F00000780000700023800024
:10AFD0003C00003000002000002000003C00003F4A
:10AFE000E00023F80000E0002700003E00003FE002
:10AFF0000021F80001E0003E0000200000000000F9
:10B000002008002008003838003E68002780000330
:10B01000C8002CF800383800201800200800000074
:10B02000000000002000003003003C01003F8300CE
:10B0300023EC000070002380003C00002000002072
:10B040000000000000000000000000380800203868
:10B050000020F80023E8002F88003E080038080090
:10B060002018000070000000000000000000000038
:10B07000000000000000000008000014001FF7FCA2
:10B080003000062000020000000000000000000068
:10B090000000000000000000000000000000FFFFB2
:10B0A000FF000000000000000000000000000000A1
:10B0B0000000000000002000023000061FF7FC0026
:10B0C0001400000800000000000000000000000064
:10B0D00000000000000000180000600000400000B8
:10B0E00040000020000010000008000004000004E0
:10B0F00000000C0000100000B5E702000200020092
:10B100007FF0421042107FF0421042107FF0420068
:10B110000208020801F800000000D7D37FF00020E9
:10B120000040008001000200FFF80200020002005F
:10B130000200020002000E0000000000BCBC102053
:10B140001020102013FEFC201020102015FC188465
:10B150003088D04810501020105051882606CAF56B
:10B1600001000120011001107FFC03800540054013
:10B170000920111021084104010201000100010011
:10B18000D2BA0080404027F81140014082784248FE
:10B1900016A81AD0235022204220425002880000D4
:10B1A0000000BEA73FE020203FE020203FE000005D
:10B1B000FDF885088508FDF885088508FDF88508EF
:10B1C00000000000B2E200084F8828880AA88AA878
:10B1D0004AA80AA82AA82AA8422845088488888854
:10B1E000103800000000CAD44050204820400FF81A
:10B1F0000040E04027402240224022202A2833A855
:10B200002E18000800000000B3CC00001BF0E21074
:10B21000221023F0F800200033F068806080A3F053
:10B220002080208027F800000000D0F202000100FA
:10B230003FF820002FF02020224021803FF8208876
:10B24000209040804080838000000000D1D5200005
:10B2500010F87E20444028F87E8848A850A864A8AA
:10B2600048A872A884501888610800000000C9AB83
:10B27000100010003FE0404080807FF042104210FC
:10B2800042107FF04000400840083FF800000000F6
:10B29000CCEE20802FF8208027F0F41027F0241027
:10B2A00027F0241027F03410CFF8022004100000FB
:10B2B0000000B3E404000200FFF808001040202062
:10B2C0007FF0089008800880088010882088C07867
:10B2D00000000000CEC4040002000200FFF810408D
:10B2E00010400880088005000200050008803060DA
:10B2F000C01800000000D7D604000200FFF8800844
:10B3000080083FC0008001000200FFF80200020038
:10B3100002000E0000000000CFD43FE020202020DB
:10B320003FE0202020203FE008804890289028A07F
:10B3300008800880FFF800000000CABE00003FE05F
:10B34000000000000000FFF802001240122022104E
:10B350004208820802000E0000000000CDBC7FF809
:10B360004008440847C84848548843084CC87338C4
:10B3700040884C08430840887FF800000000C6ACB5
:10B3800000802080208020803FF0200020002000CE
:10B390003FC020402040204040408040000000004E
:10B3A000B4A520403840484091F07D50555055504C
:10B3B0007D5055F054407C40545057F88C080000A4
:10B3C0000000C3FE2220222027F8FA2027F02410B4
:10B3D00027F03410E7F020802FF821402220EC18CD
:10B3E00000000000CAE440804140F22044108BE895
:10B3F000A000F78824A827A834A8E7A824A82488B0
:10B4000025B800000000C8EB08000400040002009A
:10B410000200050005000880088010401040202030
:10B420004010800800000000C8AB020002000500C8
:10B43000088010402020DFD8020002001FC0020058
:10B4400002000200FFF800000000B3CC00001BF077
:10B45000E210221023F0F800200033F068806080B2
:10B46000A3F02080208027F800000000BCBC2080D2
:10B4700020802080F7F02080208027E03220E2200A
:10B480002140208021402220EC1800000000CAF555
:10B490000200024002200200FFF807000A800A8032
:10B4A0001240222042108208020002000000000028
:10B4B000D6A702000200FFF8020002007FE0102081
:10B4C0001040088005000200050018C0E0380000A8
:10B4D0000000B3D62080208023F0F880208027F859
:10B4E00028203020E7F82020222021202020E0E022
:10B4F00000000000D7A8020002007FF00400040052
:10B50000FFF8080010003FE0002000401C8003000E
:10B51000008000000000D7A201004080200017F04A
:10B52000008080804080008017F010802080208084
:10B5300040804FF800000000C5FA2040244024401D
:10B54000F4482450276024403440E4402440244000
:10B5500025482648E43800000000B7A20200222057
:10B56000221044007FF8040008000FE0142024405B
:10B570004280810006C0383800000000B3C900A036
:10B58000009000807FF8408040907C90449044A0E0
:10B5900044A0444858A84118820800000000B9A6F9
:10B5A00001000100F90023F02110211021102110C9
:10B5B00021103910C21002100410086000000000B1
:10B5C000D2C60000002000780CE4790451681030E5
:10B5D0007E6019981A3C2FE448E408380030006077
:10B5E0000000D1A100000120012003FC62203420D2
:10B5F000042003FC240021B021202220323E180028
:10B600000FE00000D4F10000000010FC1304110C46
:10B610003DF8703E10D015907CF0503E18101BFE87
:10B62000023000200000CFEE0000000003FE0060AA
:10B630007C4012FC11041106113611241F44794478
:10B6400000C0009C01860000C4BF000000000FE0A5
:10B650003C18200820043E04600460047E0460045A
:10B66000200C20081FF001800000B6CC000008006C
:10B6700011FC103E3EF82D8C2904490409043E8C2F
:10B6800050FC10881EC811FC100E0000B0B4000061
:10B690000040006012FE13023A427F4410C41BFEB9
:10B6A0003C987190113011A00078004C0000C8B790
:10B6B0000000004000F878C41F8C313821EC2126AE
:10B6C000413A7DE2272225FA3D26012401040000AB
:10B6D000B6A80000010001705FFC700420042FF880
:10B6E00001001100113821C431003F0063E04038EF
:10B6F0000000B3A4000000000818086008C00B0098
:10B700001E00181C7FF01000118010E01838098E00
:10B710000F000000B0B400000040006012FE1302F1
:10B720003A427F4410C41BFE3C987190113011A026
:10B730000078004C0000B7B50000000007F80600D4
:10B74000240014F8078C04042408261825F0647CCF
:10B7500064C220801FC00000BBD8000000001FF0A2
:10B7600030182008278C2C44284428442CC42784D3
:10B770002004300C1FF803800000C7B60100210828
:10B7800021083FF800202220223EFF42229422106E
:10B790003E10221022283E2822440082CABD0048C2
:10B7A000004400440040FFFE004000403E4008408E
:10B7B0000840082008220F12780A20060002BFAABB
:10B7C00000007FFC08200820082008200820FFFE39
:10B7D00008200820082008201020102020204020C9
:10B7E000B7A201001110110822003FFC0200040062
:10B7F00007F80A080908111010A0204040A00318FB
:10B800001C06CDF800007FFC400440044214529412
:10B810004A54442444244A544A54529461044004EF
:10B8200040144008D6D001000100010001003FF89B
:10B83000210821082108210821083FF821080100DA
:10B84000010001000100CEC4020001000100FFFE62
:10B85000101010100820082004400280010002800F
:10B86000044008203018C006B2E2000427C4144483
:10B870001454855445544554155415542554E554D1
:10B8800021042284224424140808CAD40028202435
:10B890001024102007FE0020F02017E011201110C6
:10B8A0001110151019CA170A020600020000000044
:10B8B0000000000000000000000000000000000088
:10B8C0000000000000000000000000000000B4F3D1
:10B8D0000000000000000018000010000010000030
:10B8E000100000100000100C3FFFFE0010000018B8
:10B8F0000000180000340000340000220000620044
:10B9000000410000C1800080C001006006003808CE
:10B91000001C300000000000D4BD0000000000004A
:10B920000300C00200B00200980260881F888C02E9
:10B930000FF0020C80022C887FDC88030C901B0C1B
:10B94000D01B0C6013EE60131E64130CF413019CE7
:10B950001B020C27040421D800407FFC4007F8009C
:10B960000000B4B400000000000003800803000CD5
:10B9700002E00C06300C04198C08088C08008C18A6
:10B98000208C2FF08C48208C08208C08208C0820DC
:10B990008C08608C09C10C08080C08080C08080CFD
:10B9A0000C0C0C07FC78000010000000D0C2000056
:10B9B0000000000002000801003C0133C03EC2004C
:10B9C000086200044200048200049A0C3FFFFE015A
:10B9D00002300102300112301FE2300102300D420C
:10B9E000301936301114302114302108304710300E
:10B9F000022030000000D2BA000000000000000663
:10BA0000001803000C020C04FDF001198001110064
:10BA10004233083222F812421812651004E49005ED
:10BA20006AB0056A200A71200861403860C0186059
:10BA3000C018616018623018641E087800000000A9
:10BA4000BEA700000000000001004001FFC001008F
:10BA50004001004001FFC001004001004001FFC063
:10BA60000100400000001064081FE7F810460810AD
:10BA700046081046081FC7F810460810460810462A
:10BA8000081FC7F8104608000000C6C100000000EB
:10BA900000000800000FFFF80C00180C00180FFF42
:10BAA000F80C40900C30C00C10800C11100DFFF8F9
:10BAB00008308008308008308808309C1FFFE01074
:10BAC0002080102080206080204080408080030003
:10BAD00080000000B2E200000000000011000C092C
:10BAE000FE080D860805864801A64841B64833B6CB
:10BAF0004813B64815B64805B64805B64805B648D1
:10BB000009A64809A64839A4481820481858081812
:10BB10004408188608190238060018000000CAD424
:10BB20000000000000000001A01001D80800880CEF
:10BB3000008804008400FFFE0000800000800400F4
:10BB4000803C0280047DC00408C004084004084012
:10BB5000044860048822050F3407381406E01C04EA
:10BB6000000E0000060000000000000000000000C1
:10BB700000000000000000000000000000000000C5
:10BB800000000000000000000000000000000000B5
:10BB900000000000000000000000000000000000A5
:10BBA0000000000000000000000000000000000095
:10BBB00000000000D4BB000800000024E8010000E1
:10BBC00042080008D0BC0008E801002468550400C1
:10BBD000FC880008113C90D00304F13210320113AC
:10BBE0000A0632022A400C13916C1408DB6B14080D
:10BBF000A56D42081A1D101A8D101AA704C11A71DA
:10BC0000181A61041A81041A510414090243130218
:10BC1000011DC0320904551A020B13052416100128
:10BC20000524011009010424020205240617010756
:10BC300005820308151009040133020A1D070501D6
:10BC4000027B2C07058107110937442A40072A8106
:10BC500007112B0907440A2204440A16FF44411322
:10BC6000897A1B08D1041AE104130D7B1B087D049B
:10BC70001A550C1A99041A1237311E408304405782
:10BC80006D24020301071B040309041A031AC225C9
:10BC90001152081BD5095C1904139D081B08ED08F7
:10BCA00013B596140889971408400D122434401FC8
:10BCB000C03230323842202E400D0424401814C0C7
:10BCC00003301AF0181CE0012008B11CFFFF1F040C
:040000050800029954
:00000001FF
